:020000040800F2
:20000000681D002019F50008DB680008436B0008FFFFFFFFFFFFFFFFFFFFFFFFFFFFFFFF34
:20002000FFFFFFFFFFFFFFFFFFFFFFFFFFFFFFFFFFFFFFFFFFFFFFFFFFFFFFFFFFFFFFFFE0
:20004000FFFFFFFFFFFFFFFFFFFFFFFFFFFFFFFFFFFFFFFFFFFFFFFFFFFFFFFFFFFFFFFFC0
:20006000FFFFFFFFFFFFFFFFFFFFFFFFFFFFFFFFFFFFFFFFFFFFFFFFFFFFFFFFFFFFFFFFA0
:20008000FFFFFFFFFFFFFFFFFFFFFFFFFFFFFFFFFFFFFFFFFFFFFFFFFFFFFFFFFFFFFFFF80
:20480000681D002019F50008DB680008436B000800000000000000000000000000000000DC
:20482000000000000000000000000000DF9100080000000000000000617A000821F2000802
:204840001FA700085FA90008ABBB0008EFBF0008F7D10008BBD3000815EF000867F1000884
:20486000FFF400080BF500083DF500083FF5000841F5000843F5000845F5000847F50008BB
:2048800049F500084BF500084DF500084FF5000851F5000853F5000855F5000857F50008B0
:2048A00059F500085BF500085DF50008BDBD0008DDD600085FF5000861F50008A3AA0008A4
:2048C000FFFFFFFFFFFFFFFFFFFFFFFFFFFFFFFFFFFFFFFFFFFFFFFFFFFFFFFFFFFFFFFFF8
:2048E000FFFFFFFFFFFFFFFFFFFFFFFFFFFFFFFFFFFFFFFFFFFFFFFFFFFFFFFFFFFFFFFFD8
:20490000000000000000000000000000000000004A2D4C696E6B204F422D53544D33324615
:204920003037322D436F727465784D20636F6D70696C6564204D61792020342032303137DD
:204940002031343A34343A303000436F7079726967687420323030332D323031342053454C
:20496000474745523A207777772E7365676765722E636F6D0000000000000000000000003B
:20498000FFFFFFFFFFFFFFFFFFFFFFFFFFFFFFFFFFFFFFFFFFFFFFFFFFFFFFFFFFFFFFFF37
:2049A000FFFFFFFFFFFFFFFFFFFFFFFFFFFFFFFFFFFFFFFFFFFFFFFFFFFFFFFFFFFFFFFF17
:2049C000FFFFFFFFFFFFFFFFFFFFFFFFFFFFFFFFFFFFFFFFFFFFFFFFFFFFFFFFFFFFFFFFF7
:2049E000FFFFFFFFFFFFFFFFFFFFFFFFFFFFFFFFFFFFFFFFFFFFFFFFFFFFFFFFFFFFFFFFD7
:204A000008B4024B9C4608BC6047C046ED05002038B4002B1FD10400503478300078002851
:204A200001D0636A17E0206A00280CD0C500E4696419083C2568AA4201D363680BE0083C39
:204A4000401EF7D107E0C0239B032068AB4A904201D1F0231B04CB600120087431BC704709
:204A6000F8B50E0004005034002332002100FFF7CFFF00220221200001F068FA0500207D5F
:204A80000106022001F0BFFA07003100052001F0BAFA38436168A94206D065600600290048
:204AA000042001F0B0FA30430500207D000610210143022001F0A7FA010029430800F2BDCF
:204AC000F8B50E0004005034002332002100FFF79FFF00220221200001F038FA0500207D5F
:204AE0000106022001F08FFA07003100052001F08AFA38436168A94206D06560040029004A
:204B0000042001F080FA2043002802D50020C043F2BD0020F2BDF8B50024BE4E356AC8358A
:204B20000021072001F0C2FA01276946072001F0BDFA0098C00C384003D1306A281AF4D585
:204B4000E4432000F2BDFCB583B007000E003C0050340A9DA80001D5012020762807000F8C
:204B600002902068654988420BD1207E002801D0012200E0039A029882403100380001F0DA
:204B800025FBFF231B042B40320021003800FFF73FFF0B98019002980090049B039A3100BF
:204BA000200001F048F90021217605B0F0BDF6B583B007001E003C00503401250A9881007D
:204BC00000D525760107090F01910A46012191407A22BA5C002A36D0039AB24B9A4232D115
:204BE000042977D10499012974D1AF493800FFF737FF00281DD40021072001F057FA694686
:204C0000072001F053FA70780002B17809040143F07800060843A54A02400098F02109032C
:204C200001401143072001F0EEF9002804D501F0DEF90020C0435CE001F0C4F900210320C6
:204C400001F034FA44E0039AB94B9A4242D1042940D1049901293DD1300001F00AFC0090B7
:204C6000B3493800FFF72CFF0028E2D10099072001F0C9F90028DAD401F0A4F9009840074E
:204C800022D5022001F005FE0021032001F00EFA00281DD05F4E306A9621C9004018019005
:204CA000A44F642001F0F5FD6946002001F0FEF9002804D1009838409F49884208D00198B3
:204CC000316A401AEDD503E00021032001F0EEF901200EE0FF231B04034021003800FFF73C
:204CE00097FE019800903300049A0399200001F0F4F80021217605B0F0BD0000FF00010E64
:204D0000F2B582B017001C000100503101916649FFF7A6FE002807D40021072001F0C6F92F
:204D20006946072001F0C2F90298007801F0C8FD009D000202210143062001F064F9B64EAB
:204D400035402900072001F05EF90198FFF7E3FE002810D4009D0021062001F0A7F939001C
:204D6000062001F0A3F92E403100072001F04BF90198FFF7D0FE002808D40298401C02909C
:204D80003F1D641ED0D1002003B0F0BD0020C043FAE7F2B582B017001C007A21415C0029A3
:204DA00004D00299FFF7ACFF06002FE03E49FFF757FE002802D50020C04328E002980178BF
:204DC000052001F020F90021042001F06FF900265A48056AC8356946042001F067F9009816
:204DE000C00305D45548006A281AF4D5F6430DE00021062001F05AF93900032001F056F9B8
:204E00000298401C02903F1D641ED7D1300003B0F0BD000078010020F2B582B017001C004F
:204E20000100503101912049FFF71AFE002807D40021072001F03AF96946072001F036F982
:204E40000298007801F03CFD009D000203210143062001F0D8F8704E35402900072001F0B4
:204E6000D2F80198FFF757FE00280CD4009D3968062001F0C8F82E403100072001F0C3F8F5
:204E80000198FFF748FE002808D40298401C02903F1D641ED4D1002003B0F0BD0020C0438B
:204EA000FAE70000FCED00E0F0ED00E0FFFFF0FFF2B582B017001C007A21415C002904D05D
:204EC0000299FFF7A9FF06002EE09349FFF7C8FD002802D50020C04327E03968062001F00D
:204EE00092F802980078802149020143052001F08AF80021042001F0D9F800260F48056A5B
:204F0000C8356946042001F0D1F80098C00305D40A48006A281AF4D5F64305E00298401CF8
:204F200002903F1D641ED8D1300003B0F0BD00000CED00E0FF0F00007704000078010020CD
:204F4000F0B583B007003E00503600247249FFF787FD05007A20385C002825D0002D1ED4E6
:204F60000021042001F0A2F8050001A9072001F09DF80095050002A9072001F097F8010018
:204F80002943009D29430D0009D40198800302D57A203C5404E002980403E40F00E0E44316
:204FA0007A20385C002833D10021042001F07EF804002C4301A9042001F078F8204315D5FC
:204FC0000020706054493800FFF74AFD05000021042001F06BF804002C4301A9042001F0FF
:204FE00065F8204302D50020C04312E0019800030BD54A49042001F006F80021042001F0AD
:2050000055F801A9042001F051F801988403E40F200003B0F0BD0000FFFFF7FFF1B582B0DC
:20502000044679346078002842D03B490298FFF717FD0021072001F039F86946072001F00E
:2050400035F800980103C90F07D1C0218902014300910099072000F0D6FF0021072001F0D8
:2050600025F82F4F3D6AC83501A9072001F01EF8002802D50026F64308E001980603F60F2C
:2050800002D1386A281AEFD501980090002E0CD1002060700098234901400091072000F084
:2050A000B2FF0021072001F001F8607800282ED119490298FFF704FD2078C000174D054317
:2050C0002900072000F09FFF01F040F8144F3E6AB61C01A9072000F0E9FF002802D5002024
:2050E000C04306E001998803C00F02D1396A711AEFD506002078002809D008208543290056
:20510000072000F080FF0021072000F0CFFF00202070300003B0F0BDF0ED00E003005FA0F4
:2051200078010020FFFFFCFFF0B58BB00400CA07D20F04928807C00F69460873206DCA4989
:20514000884218D1200001F067F8002802D50020C04387E1200001F059F8C4492000FFF71D
:20516000AFFC002807D40021072000F04CFF002801D100F027FF6846007B002873D06846AC
:2051800000210173BA492000FFF79AFC80202058883000680125284202D0A843019005E0D0
:2051A00000F0D4FF01A9032000F080FF01993031052000F028FF00F0C9FF01A9032000F044
:2051C00075FF019800284ED00021C94388424AD0A8430190014610392000FFF771FC0021BB
:2051E000072000F063FF06A9072000F05FFF01990C39052000F007FF0021072000F056FF8B
:2052000006AE311D072000F051FF01990839052000F0F9FE0021072000F048FF3100083155
:20522000072000F043FF0199091F052000F0EBFE0021072000F03AFF0C363100072000F05A
:2052400035FF06988B4988420DD107988A49884209D108988949884205D10998884988429C
:2052600001D16846057387492000FFF729FC1F21072000F0C8FE844F39002000FFF7F0FB01
:205280000021042000F012FF6946072000F00EFF02A9072000F00AFF00200099890303D40E
:2052A0000299090300D50120260079366946097B002956D0002800D099E0B078002827D141
:2052C00072492000FFF7CCFB0021042000F0EEFE05A9042000F0EAFEFF2505992943042019
:2052E00000F091FE0021042000F0E0FE01A9042000F0DCFE01980540280001F0AEF8019056
:2053000008200199401AB0700599042000F07BFE39002000FFF7A4FB02985D490140802017
:205320004002084302900146072000F06CFE009880B2009000200490564C00980107C90F5E
:2053400007D008218843009001462143042000F05AFE009807218843009004432100042034
:205360004DE0012500284DD0B94F0098384005430095484C29462143042000F044FE049847
:2053800000282DD0009802210143009100992143042000F038FEAF48056A6D1D00210420DC
:2053A00000F084FE6946042000F080FE0198800303D4A848006A281AF4D5009807400820DB
:2053C0003843009001462143042000F01CFE009802218843009004432100042000F013FE46
:2053E0000298B54901400291072000F00CFE029C0121062000F007FEB0492140072000F0D4
:2054000002FE18E00498C000B9490143019104980099C9080D40A84203D00199042000F0A2
:20542000F2FD01980221884301900146042000F0EAFD00F0C7FDAF480068002801D0FFF721
:20544000DFFA00F0BFFD0021032000F02FFE6946097B7170C90701D50121F170002801D42C
:20546000049931700BB0F0BDFF00010E50EF00E008ED00E04A4C494E4B4D4F4E48414E4407
:205480004C45520030ED00E0F0ED00E020ED00E0FFFFF3FF00005FA0F0B587B00400206D26
:2054A0009549884218D1200000F0B6FE002802D50020C043C9E0200000F0A8FEB4492000F9
:2054C000FFF7FEFA002807D40021072000F09BFD002801D100F076FD26007A36AD4D307836
:2054E000002800D184E0AC492000FFF7B9FA0021042000F0DBFD04A9042000F0D7FD049853
:20550000C0B2049029002000FFF7AAFA002807D40021072000F0CAFD6946072000F0C6FD17
:2055200000988021C902014300910099072000F06AFD684614210173012305AA03A9200085
:20554000FFF7DEFBAF4F0598384001900146049A0120082375785B1B9840101800020843F7
:205560000190012301AA03A92000FFF755FC009D0121062000F047FD50492940072000F086
:2055800042FD0021072000F091FD324D2E6AC83602A9072000F08AFD002802D50020C04386
:2055A00008E002990803C00F02D1296A711AEFD502990091050041D40098A349014000913D
:2055C000072000F020FD012301AA03A92000FFF797FB019807400598FF210902014039430F
:2055E0000191012301AA03A92000FFF715FC25E029002000FFF764FA9449072000F003FDE1
:205600009349072000F0FFFC00F0A0FD114D2C6AA41C02A9072000F049FD002802D5002034
:20562000C04306E002998803C00F02D1296A611AEFD505002E49072000F0E5FC00F0C2FCC5
:205640000021032000F032FD280007B0F0BD0000FFFF00007801002002B582B069460F22FB
:205660000A70012302AAFFF723FC03B000BD70B582B00400774DC04E00290ED000F0B0FC8B
:20568000002060653068A84214D26946012000F00DFD0099012081430AE03068A84209D22E
:2056A0006946012000F002FD009801210143012000F0A9FC73BD0000FFFFFAFFFFFFF7FF5C
:2056C00001290AD9091F0CD0091F04D008390AD0703904D009E0A9487047A94870471F20AD
:2056E0007047032070470120704700207047000003005FA040120020FF00010EF0B583B010
:2057000005000F002C00503420689E4988423CD1002001909C492800FFF7D2F9002807D4FD
:205720000021072000F06FFC002801D100F04AFC964E0023320021002800FFF769F900209C
:20574000009001AB01223100200000F0BFFB0198C004840D641C01980001450C6D1C0126E6
:205760000320019A0240921C012191403E603871880000F0DBFEF871280000F0D7FE7871B1
:20578000200000F0D3FEB8713E74002003B0F0BD50EF00E0F0ED00E020ED00E0F0B583B02C
:2057A00005002C00503420687649884201D0002026E0B04E0023320021002800FFF728F979
:2057C0000020009001AB01223100200000F07EFB012701984008384012D0C14E00233200C9
:2057E00021002800FFF714F90020009001AB01223100200000F06AFB0198000C0740380014
:2058000003B0F0BDFF00FFFF38B5046D5D4DAC4217D1049CA4000919CC79A240202489797A
:20582000611A8B4013431C00AE49FFF749F9002807D42100072000F0E6FB002801D100F07B
:20584000C1FB002032BD0000FFFFFBFF0F005FA00D005FA0A6AE0000F5B585B00E00842A7C
:2058600002D20020C04385E0300050300190059840690290059880690490842200213000A2
:2058800000F014FE059800680090002801D1964800900098000E954CFF2808D0032801D087
:2058A0000E2804D100983749884200D0904C0598007B694608730598407B01061BD500219D
:2058C000820701D580218903420703D50A008021C9031143020703D50A0080210904114363
:2058E000800603D40800802149030143301D01677820012131540598807B002804D0202842
:2059000002D201248440641E351D0498042809D3029800F0AEFDE8660298001DA866E96EB3
:2059200001F00EF937002C378020400000F0FEFD2021785420370520787036606D48686086
:205940006D4828600020E86028616C49A96001996A46127B0A75019901228A7501998C60C3
:205960000199009A0A600199486078360598B0600698843807B0F0BD3C1200203700008009
:2059800001000080FF00010E84ED00E080ED00E030B5C5B005000221684601F0ABF9684667
:2059A000018835A801F0A6F968460088042804D335A800F05EFD040000E04B4C9022002142
:2059C00001A800F073FD019401A80121017100214171017325A805904AA00890402225A991
:2059E00001A8FFF739FF01210598FFF740FE642D12D0652D14D06E2D16D06F2D18D0792D49
:205A00001AD07A2D1CD07B2D1ED07C2D20D0822D22D0832D24D026E001A801F089FA22E070
:205A200001A801F0FDF91EE001A801F03FFB1AE001A801F067FB16E001A801F089FB12E008
:205A400001A801F09CFB0EE001A801F0A1FB0AE001A801F0ADFB06E001A801F0B2FB02E0B6
:205A600001A801F0E9FB00210598FFF700FE45B030BD000078ED00E070B582B006690124E4
:205A800001207C21715C002929D01D493000FFF717F805000021072000F008FB0100294311
:205AA0000D006946052000F001FB284316D40098C00C204003D07C36002030700EE0009835
:205AC000000C04400AD10098802149020143072000F099FA6946052000F0E8FA002076BD30
:205AE00014ED00E074EF00E0FF000003FF030000FF0F00009D570008FD56000809580008B0
:205B0000FCED00E000000000DD680008036A0008934D0008B14E0008295100089954000894
:205B20001D500008414F0008000000005956000859580008474B0008AF4B0008000000004C
:205B4000C15600080000000000000000000000006F560008795A0008F4B584B005000E008E
:205B60001F0000200290B80701D101200290287E421E9241D20F0221280000F0E7F9040037
:205B8000287D0106022000F03EFA00903100052000F039FA009908436968A14206D06C60CC
:205BA00005002100042000F02EFA2843002856D100F0CCFA002852D10498022847D3441E86
:205BC0000A9E0298002826D0002E07D0F068B168401A844200D82000009000E000940025AE
:205BE0003900072000F062FA002836D13F1D6D1C00988542F4D3002E09D0B06800994018AF
:205C0000B060F168884202D33000316888470098241AD9D11BE001A9072000F047FA00283F
:205C20001BD101983870010A7970010CB970000EF8703F1D002E08D0B068001DB060F16897
:205C4000884202D3300031688847641EE3D101A9032000F02BFA002804D000F0C8F9002028
:205C6000C04304E00199380000F0EEFB049805B0F0BDF5B583B00E001C00007E421E9241DC
:205C8000D20F0A9F3900039800F060F905000398007D0106022000F0B6F900903100052092
:205CA00000F0B1F90099084303994968A94208D003994D6000902900042000F0A4F900990A
:205CC0000843002835D100F041FA002831D10498022828D3451E0120B84002906846032155
:205CE000C91B017001A9072000F0E0F9002802D000F07DF91DE001986A4612783240D10042
:205D0000C840019001982070641C002F03D00198000A2070641C0398007E002801D10298DF
:205D200036186D1EDED101A9032000F0BFF9002802D00020C0430FE001980321C91B314048
:205D4000C900C840019001982070641C002F02D00198000A2070049805B0F0BDF3B583B02B
:205D600015001C000A9F012F01D1924804E0022F01D1914800E0012001900398007E421EA2
:205D80009241D20F7910039800F0E0F806000398007D0106022000F036F9009004990520AB
:205DA00000F031F901000098014303984068B04209D00398466000913100042000F023F9AB
:205DC00001000098014300290CD1A00710D1042F0ED12168072000F016F9241D002804D555
:205DE00000F005F90020C04323E06D1EF1D119E02178022F0CDB0A00607801021143032F2D
:205E000006DB0A00A0780004E17809060143114301984143072000F0F6F80028E0D4E41980
:205E20006D1EE5D100F0CEF80021032000F03EF9002005B0F0BDF9B581B00D001600807D7F
:205E4000002802D10020C0433EE0002708980890099809900BE02000089988400199097ED8
:205E6000002900D12D18029908180290361B002E29D001988068A8430899C840401C019913
:205E8000097E002901D0340003E03400864200D904000898022808DB09980090029B2200F4
:205EA00029000198FFF758FE06E00090029B220029000198FFF7DDFE002801D5070002E025
:205EC0003F18A042C7D0380003B0F0BD10B582B0049C0094FFF740FE16BDF9B583B00D003A
:205EE000160000270A980A9001200A99884001900CE03F190A99200088400399097E0029F1
:205F000000D12D18049908180490361B002E1AD003988068A8430A99C840401C0399097E19
:205F2000002901D0340003E03400864200D9040001980090049B220029000398FFF70EFFC6
:205F40000028D6D50700380005B0F0BD78B403681A4CA34201D1012300E0002380256D04DC
:205F6000C468E60201D48225ED05260203D52E0080252D053543660203D52E008025ED041E
:205F80003543A60203D52E008025AD043543240305D5007C002802D12800094D0540002BA7
:205FA00003D128008025AD05054329431001084372BC70470101010101000100FF00010E85
:205FC000FFFFFFF380B56846FF21417000210170082300AA921C6946401C01F064FC01BDEE
:205FE00000B583B0754830236A46010006E000B583B0724830236A4601000831103001F002
:2060000052FC03B000BDF0B58FB0002200240B0C4B401D0A5D402B096B409D085D4003917D
:206020006B086B40D907C90F03AB1971644F3E6A6436644D69462818007A08704A7009E028
:2060400084235B0005AA290010312800343001F02AFC641C0D2301AA69462800603001F0CF
:2060600022FC01A840784007400F012808D1212301AA03A96835280001F015FC002013E094
:2060800002280CD0042802D1FFF7AAFF05E0022C03DA4D4800780028D2D0002003E0386AF0
:2060A000301AD7D50120C0430FB0F0BDF2B58EB00021002502AA1171424E01AA305C1070BA
:2060C00051703F48076A643709E084235B0004AA310010313000343001F0E5FB6D1C0D2343
:2060E0006A4601A93000583001F0DDFB684640784407640F012C13D1C006840F21236A4643
:2061000002A95A36300001F0CEFB0E98002804D00098800004430E98046000200FB0F0BDC3
:20612000022C0DD0042C02D1FFF75AFF05E0022D03DA254800780028C7D00020C043EDE776
:206140001F48006A381ACAD50120F7E780B500210720FFF7ABFF02BD00B58BB019488423AA
:206160005B0001AA01001031343001F09CFB69460020FFF79BFF002811D469460120FFF7B9
:2061800095FF0098B22101400BD0FFF729FF69460120FFF78BFF0098A021014001D00120EA
:2061A00009E0A021C90500910120FFF72CFF401E8041C043C00F0BB000BD00009002002079
:2061C00078010020A8020020601B0020F8B403008818401E1F22D24311400240501A420976
:2061E000521C49090124C9B2C8081D182C20285C01264F077F0FBE4006432C352E70491CB4
:20620000521EF0D14E331C70F1BC704700B520212C3001F00BFC00BDF1B588B04E30007801
:20622000002800D1B8E008984E300021017008988168080000D1AFE008980068884700282D
:2062400000D1A9E008984268100007D008991831089800689047002800D59AE00898016969
:20626000080005D0089800688847002800D590E00020039008980190012405E00398401C18
:2062800003900198001D0190039808998969884276DA0198007F022803D0032801D004289F
:2062A000ECD10198C07F08994D310978401A0490002008994C310978019A527F8A4200D2F2
:2062C000881A00210291049901228A40069201218140059118E00898C66830000AD0039862
:2062E00000902B00029A0899183108980068B04700284ED46D1C0198817F01208840854242
:20630000E9DB0298401C029002990198427F012090408142B2DA08460499884008994C312B
:206320000A7801219140491E0140002205980128E7DB03460800069D012D0CDBC608089F18
:20634000BE192C36367847077F0F3E41264002D1401C6D1EF2D1921910D10198407F049D93
:2063600045190120A840081808994C310D780121A940491E01405B1EC3D0DBE70025BAE7AC
:2063800008984169080007D0089800688847002802D50020C04300E0002009B0F0BD38B489
:2063A000012100220368001D002B0BD00468001D0C4202D04D466D1E64192260241D1B1FCA
:2063C000F0D0FAE732BC704701680A060B0A1B061B0A13430A02120E12021A43090E114345
:2063E000016070470106020A1206120A0A430102090E09021143000E08437047CA088218FC
:206400004807400F9107C90E4118032082431068002906D0C840030050682022511A88407F
:206420001843704702681170090A5170921C0260704702681170090A5170090A9170090ADE
:20644000D170121D026070470170090A4170090A8170C01C090A01707047010006D000206C
:2064600001E04908401CCA07FBD570470020C04370470178427812020A438178090411436E
:20648000C07800060843704718B4012A0BDB0300401C0C00491C1B782478A34201D0012009
:2064A00002E0521EF3D1002012BC7047012A03DB0170401C521EFBD1704778B40300002009
:2064C000002480252D0601E03100641C294202D14E00B342F8D2002C09D440008B4203D3F7
:2064E0005B1A0500012028434908641EF5D5002A00D0136072BC704780B56A46FFF7DDFFF0
:20650000009802BD80B50022FFF7D7FF02BD80B5002807D5002243421800FFF7CEFF010086
:20652000484202BD0022FFF7C8FF02BD002101E0491C4000002800D4FAD11F20401A7047B6
:206540000278401C0B78491C002A01D09A42F7D0D01A704738B472B6A54A906800211171A0
:2065600062B6002823D00168002920D043694C699C421CD100E021000C68002C02D06569F9
:206580009D42F8D072B603681469844200D11361026A13601A6201620A680260002A00D0AD
:2065A0001062086038200A00393212780A5462B631BC7047F8B500278D4C6770012020705B
:2065C00072B6E06B010004D08047E76367633820275462B601F02CFA0078CD2802D07D20BA
:2065E00001F02CFAA068002807D0C16B002904D009680A0001D0406888473120205C00289C
:2066000009D0A06838303021615C01702079002801D0FFF79FFFA068002805D0017C0029E1
:2066200002D1416B491C41632069002826D002E02868206162B672B62569002D41D02E7C82
:20664000002E3ED070070FD5E868216A411A012906DA280000F090F8287C002804D10DE035
:20666000616A411A00D56062FB2030401028DFD1A86880684068007C0028D9D172B620E0D4
:206680002069002804D0686921694969884218D3287C400710D5E868216A401A012806DAA5
:2066A000280000F069F872B6287C002809D0E868616A411A00D5606262B62D68002D72B685
:2066C000DED1607900280BD12069002832D02069007C0028206911D08068806840680DE07F
:2066E0006771206A8021C90540186062E169080001D02000884762B6E568DFE7A060C06A48
:206700000078CD2802D0782001F098F9A068C16B002904D049680A0001D040688847A068E4
:206720003030017A3022A1543122A1540168491C016006E03120275430202754A7602770A5
:2067400062B62000F2BD10B5294C2078401E2070207800280FD1606800280CD072B606D028
:2067600001202070200001F0D7F9002020706078002800D162B610BD38B581681C4C0029BA
:2067800009D0226AC2600A684968002A00D051600A6000218160017C8907890F017413D13A
:2067A0002169002911D1206101202178002906D12070200001F0B0F90020207000E060715E
:2067C0006078002800D162B631BD42694B699342E9D38142E8D09A42F6D103001B68002B23
:2067E000EED05D69AA42EBD18B42F7D1DBE700007801002038B54169304C2278521C2270D0
:2068000022000C3200E01A001368002B02D05D69A942F8D3036002621060002B09D0186275
:206820005A698A4202D13921415C00E0002138228154017C002906D172B6FFF79DFF6078C0
:20684000002800D162B6FFF77EFF31BD38B51B4C25782078401C2070200001F05DF9257055
:206860006078002800D162B631BD10B501F082F912480121017001F0DBF8040001F0DCF896
:20688000021B203A012A03DBCD212000FFF70EFE10BD80B509490A6A80180A78002A04D088
:2068A00062B60A6A121A07D5FBE772B68968C86004200874FFF7CAFF01BD0000780100206B
:2068C000402801D32B3806E0212801D1142002E0142800D11320C0B27047FEE7FDB584B0CE
:2068E0000D0014469549194002910C9E0D980D90E80715D5002C13D00D9801900298009033
:2069000033000122290004980069049FFF693F6BB847002873D4241A01286ED1761C6D1C0F
:206920000698400057D4A80718D5022C16D30D980190029801210143009133000122290055
:2069400004980069049FFF693F6BB847002856D44100641A012850D1B61CAD1C06980028C2
:206960001CD4042C1AD3A00803900D98019002980221014300913300039A29000498006909
:20698000049FFF693F6BB847002838D48100641A0399884231D1880036182D18022C1AD372
:2069A000600803900D98019002980121014300913300039A290004980069049FFF693F6B62
:2069C000B84700281BD44100641A0399884214D1480036182D18002C0FD00D9801900298E1
:2069E000009033002200290004980069049DED692D6BA847002802D4241A0598001B07B05B
:206A0000F0BDFDB584B00D0014464C49194001910C9EE80713D5002C11D000913300012287
:206A2000290004980069049FFF697F6BB847002800D581E0241A01287CD1761C6D1C069869
:206A4000400067D4A80716D5022C14D3019801210143009133000122290004980069049F55
:206A6000FF697F6BB847002866D44100641A012860D1B61CAD1C0698002830D4042C2ED3B4
:206A80000498C069876B38000FD0019800280CD100903300A208290004980069B8470028C8
:206AA0004AD48000241A2D183618A008029016D001980221014300913300029A2900049822
:206AC0000069049FFF697F6BB847002834D48100641A029988422DD1880036182D18022C7E
:206AE00018D36008029001980121014300913300029A290004980069049FFF697F6BB84730
:206B0000002819D44100641A0299884212D1480036182D18002C0DD00198009033002200F7
:206B2000290004980069049DED696D6BA847002802D4241A0598001B07B0F0BD0000FF3FD3
:206B40007047FEE7F8B50C0006009C4D2868002804D13000EA68D2699047F1BDAB68002BE4
:206B600018D06968CF1ABC4200D22700002F11D03A003100C01801F00BF8A868C119A96042
:206B8000F619E41B1FD02868EA68D26990470020A86001E0002C16D06868401EC74327404A
:206BA00007D039003000EA68D2699047F619E41B09D022003100A8682B68181800F0E8FF4D
:206BC000A8680019A860F1BD002804D00021002206C00838016070478E4801210170704759
:206BE000002900D1704780B5002803D08A4AD2685269904701BD70B505000C00864E3068B4
:206C0000002806D1F068406A8047706001F024F8306021002800FFF795FF70BD01B5042164
:206C20006846FFF7E8FF01BD70B588B004002022C9B26846FFF73AFC774D212C01D32026E8
:206C400000E026002868002806D1E868406A8047686001F001F8286031006846FFF772FF5E
:206C6000A41BEAD108B070BD30B589B004002022C9B26846FFF71AFC212C01D3202500E0D6
:206C8000250029006846644AD26852699047641BF2D109B030BD80B50021FFF7E5FF01BDA8
:206CA00080B55D4AD2689269904701BD01B501216846FFF795FF01BD01B502216846FFF7E3
:206CC0008FFF01BD01B504216846FFF789FF01BD10B5514C2068002808D0A168002905D0B2
:206CE000E268526990470020A06010BDE068006A804710BD80B5002901D1002002BD464AE6
:206D0000D2689268904702BD50B589B00400212C01D3202600E0260031006846FFF7EAFF3C
:206D2000002801D1A41BF2D109B050BD80B53A4AD268D268904702BD80B50421FFF7DAFF25
:206D400002BD10B582B00400684600220260FFF7D1FF69460A784B781B0213438A78120402
:206D60001A43C97809061143216016BD80B52A48C0680068804702BD80B52748C06840688D
:206D8000804702BD10B50D4C2000103000F0AEFF01F035F82148E06010BD80B51E481030E3
:206DA00001F002F901BD80B51A48002101701A48C0680069804701BD00000000300B00202D
:206DC00080B501F0D7F802BD10B582B0040004E002211148103001F00DF901F0CBF8002891
:206DE0000BD001F0C2F8012807DB0B480B49C16001212000FFF77EFF16BD01F0BBF80028E6
:206E0000E6D00021684601F09FF80028E0D50020C04316BD641B0020300B00203CF4000860
:206E2000F1B58AB00024E443082108A8FFF762FF089806900998010C0904079180B20590A7
:206E4000019000F0FAFE0599814200D90100029108469349884202D3FF218843029002980B
:206E600000F0FAFE0490002803D13EE00698001906900198002801D1059C3EE006460298F7
:206E8000864200D906000198801B0190069F002531000498FFF74AFF0395FFF767FF311A71
:206EA000039A8C1A002803D0402CF6D33F208443002D0ED1049988180090079B2200390063
:206EC0000A98C569AD68A8470500A54200D100253F19039800190390B042DED1002D02D0BD
:206EE0000024E44301E03400C0D50198002801D0FFF70AFF0498002802D0049800F0D2FE1A
:206F00002000FFF7DFFE0BB0F0BD38B50500AC683F2084430BD0210028696A681018FFF76D
:206F2000BFFE286900192861A868001BA86031BDF1B592B0082106A8FFF7DCFE069F07986D
:206F4000010C0904059180B20490044611280ED300F073FE03900498001D0399884200D272
:206F60000390039800F078FE0290002803D10DA8029014200390039E361FA64205D249489B
:206F8000864203D3760A760200E0260046480890802080000B900298099000200A900C90EB
:206FA00008A8019002980090059B320039001298C5696D68A84705000C98012D02DA241ACE
:206FC0001FD121E07F19641B291A0091002C0ED1049902984019FFF737FA0099091D0C98B0
:206FE000029A1018FFF75CFEFFF772FE0FE0029A1018FFF755FEFFF76BFEB542BBD004989E
:20700000051B2000FFF747FE2800FFF75BFE02980DA9884201D000F045FE13B0F0BDF0B54B
:20702000D3B0040005216846FFF764FE6D46297802A8FFF75FFE687800281ED0A87800280E
:207040000DD0A54E316A0F182069E169096A8847002808D1306A381AF6D5002003E0206945
:20706000E169096A88471290012808DA1298012810DB28788100091D0DE0012012902B787F
:2070800012AA121D02A92069E469E468A0470028ECD51290042112A8FFF7A2FD53B0F0BDA2
:2070A00001100000010400000B6F000870B5D4B0060002E001A8FFF793FD002442AD012143
:2070C0006846FFF717FE68460078FF2806D0684600782870641C6D1C402CF0D1230001AA12
:2070E00042A93069F569ED68A847A1006A461278FF2ADFD101AA5050091D01A8FFF770FD39
:2071000054B070BDF0B5D3B00700002442AE02AD0BE0042101A8FFF7EDFD684600783070ED
:2071200001982860641C2D1D761C01216846FFF7E1FD68460078FF28EBD1230002AA42A96B
:207140003869FC692469A047FFF7BCFD53B0F0BD10B582B0040001216846FFF7CBFD68461F
:2071600001782069E26952699047FFF7ABFDA06D002803D00121200001F09FF813BD80B5BB
:2071800001000869C96989698847FFF79BFD01BD10B504002069E169C9698847FFF792FD1C
:2071A000A06D002803D00021200001F086F810BD80B501000869C969096A8847FFF782FDBA
:2071C00001BD10B584B004000020039014210291019004E06846017803A8FFF78BFD012192
:2071E0006846FFF787FD6846007800280AD1039B019A02992069E469646AA047FFF762FD8A
:2072000004B010BD012100A8401CFFF773FD684640780128DED00AD3032804D007D26846C1
:20722000017802A8D9E76846017801A8D5E768460078FFF769FDD2E710B584B00400002087
:20724000039001200290019004E06846017803A8FFF750FD01216846FFF74CFD6846007829
:2072600000281FD103992069E269926A90471A480178491C01700120FFF70BFB01992069C2
:20728000E269526990470298FFF703FB2069E169C96988470400FFF756FA2000FFF712FD40
:2072A00004B010BD012100A8401CFFF723FD684640780428C9D00AD3062804D007D2684680
:2072C000017802A8C4E76846017801A8C0E768460078FFF719FDBDE778010020FDB584B014
:2072E0000291049D1035296903916846848A0C980C90AE8A06411ED02700B44200D9370059
:207300003A0082400092029800F042FCF61B0C98310081400191002E06D00A460098039956
:207320000918286900F034FC0198A8820098029908180290E41B9E48006A6946098B4018E9
:207340000390002C1BD00C9801906846008B00906846838A029A00212868EE68B66CB0470E
:20736000002800D50020241A0C99884002990818029003988E49096A401A0128E1DA0C9831
:20738000E88204988C30012101706846808A001B07B0F0BD30B583B00500042101A8FFF780
:2073A000A9FC00F04AFC0199814202D300F045FC01900198052815D300F04EFC04000020F2
:2073C000009000230198021F92B2211D2800FFF785FF2060011D2000FFF702FC200000F05A
:2073E00061FC02E00020FFF76DFC03B030BDF0B585B00700082103A8FFF77CFC03AC2088B5
:207400008000E188884200DA0800001D00F024FC0500E18809D10800FFF776FC65480290B3
:20742000042102A8FFF7DCFB33E0002901D0FFF761FC0026607900280AD1022000906388B1
:207440002288291D3800FFF749FF0290064614E0012810D102203885238801906088009057
:20746000E0888010C01A80002A1801213869FC69A46CA04700E0C048029002992800FEF727
:20748000E3FFB100091D2800FFF7AAFB280000F009FC05B0F0BD10B582B004000121684626
:2074A000FFF728FC684601782069E269D26B9047FFF708FC13BD1CB5040008216846FFF737
:2074C00019FC00200099012905D1019901220A438834226000E0A848FFF7F4FB13BD10B54C
:2074E00003000120002900D0C148002B5CD05968002902D00100022008439968002902D0E9
:20750000010004200843D9680C0002D00400082020431C69002C02D00400102020435C696E
:20752000002C02D00400202020439C69002C02D0040040202043DC69002C02D004008020F5
:2075400020431C6A002C03D004008020400020435C6A002C03D004008020800020439C6AAA
:20756000002C03D004008020C0002043DC6B002C03D00400802040012043002903D00100BA
:20758000802080010843996C002903D001009020C00108430100C020400208435B6C190073
:2075A00002D0010010009847FFF78CFB10BD000078010020F9FEFFFF00B583B0012100A87F
:2075C000401CFFF797FB01216846FFF793FB0220FFF79AFB00280CD101A9684640780002AF
:2075E0006A461278104300F039FF00220199FFF776FF03B000BD00B583B0012100A8401C31
:20760000FFF778FB01216846FFF774FB042102A8FFF770FB01A96846407800026A46127850
:20762000104300F01BFF029A0199FFF758FF03B000BD70B5A6B09022002101A8FEF736FFD9
:20764000012100A8801CFFF755FB01AD04E06846017801A8FFF775FB01216846FFF74AFBAB
:2076600068460078002806D101A96846807800F079FF26B070BD012100A8401CFFF73AFBD9
:20768000684640780728E2D031D3092809D002D30A280AD02BE068460178281DFFF72AFB22
:2076A000DAE768460178681DF8E768460078082802D26846047800E008242100280008309D
:2076C000FFF718FB68460078061BC5D0300000F0C3FA0690002804D03100FFF70BFB07968C
:2076E000BAE768460078001BFFF70EFBB4E768460078F9E770B582B002216846FFF7FAFAF6
:20770000684646780078C100091809014F4A541804282DDA25001035E968002928D0112E46
:2077200026D2C100081A8000494908184949096AC1602868002802D1200000F0A6FE8C202B
:2077400001212154E868C26CB00000BF43A10E5810000AD00121286890472000B0470021B0
:207760002868EA68D26C904773BD2000B04773BDFFF732FA73BD0000FAFEFFFFF8B5012085
:207780000090324F3C00324D0C358D3704262069002825D08C20205C002821D0387800282F
:2077A0001ED128682C4940182A49096A401A012816DB200000F0B4FD002800D100902000B9
:2077C00001F0F4F8002800D1009020001030C068016D080004D020008847002800D10090F9
:2077E000903490371C35761ED1D10098F2BD0000010000400100401C0022D243914201D1B6
:2078000000210420CA0052181201104B9A181369002B02D08C3200231370491C8142F1DBFE
:20782000704738B50C0000280FD4C1000818000106490D18002C03D1280000F01AFD02E026
:20784000280000F02AFD8D352C7031BDD01200204C1200207801002010270000316F0008A5
:20786000216E0008AD70000805710008517100087F71000891710008B1710008C37100089C
:207880003972000895730008977400081F700008EF730008E1830008A18D0008B77400083C
:2078A000F0B5059C02E0F0B5334C2468A6464C4655465E466746F0B4994682468B46944690
:2078C0002E4A10210420148801263602B4432304344323437446012C00DA51E04F46092F26
:2078E00000D308275C4625782D02641CA34654462678641CA24635436C0810D31A266C0A8A
:2079000000D318269153138010836D08744600BF641EFDD550837446641EFDD510E01C0C11
:20792000148010836D087446641EFDD550837446641EFDD51469640902D30124E405254387
:207940007F1ED9D14E46082E02D20824A41BE5402D0C64462570641CA4464E46092E02DBA8
:20796000083EB146BAD1F0BCA146AA46B346BC461C0C1480F0BD0000EC0A002000000048FA
:207980004F46092F00D308275C4625782D02641CA34654462678641CA24635436C0809D3D9
:2079A0001A266C0A00D318269153138010836D0850830AE01C0C148010836D0850831469B0
:2079C000640902D30124E40525437F1EE6D14E46082E02D20824A41BE5402D0C6446257075
:2079E000641CA4464E46092EBDDB083EB146C7D11206130A1A43130C1A4300BF130030B421
:207A000014001500103902D310393CC0FCD2490700D30CC000D504C0890002D30280801C08
:207A2000002900D5027030BC704700000022E5E700487047681B00206846704706490A786D
:207A4000521C0A7000224A7062B60449087008780028FCD1704700BF78010020591B00206D
:207A600038488168002901D108B00ED0EFF30982283A0368F8C243464C4655465E4678C284
:207A8000734608C2283A83685A60FEF793FD816800291CD04A68143278CAB346AA46A146CF
:207AA000984608CA9E46283AF8CA27490B60143282F3098870460421084386469069234990
:207AC000814203D02248034200D162B67047214821490968401A80F308882049C16120492C
:207AE00081610621C9438E46704701BC20461D498E4600BDFEE71C48006817490968401AF0
:207B000020380721884380F3088800210D48417062B600F012F8FEE703680CB400214170FC
:207B200062B61249124A0A6000BF72B60CBC036070470E490E4A0A6070470C490C4A0A605E
:207B40007047000078010020780100202A7B000800FF0000481D002038F5000800000001D5
:207B6000B5F20008F57A00080048000804ED00E000000010EFF3108072B604490A68FF2333
:207B80001B0413430B6080F31088704720ED00E0124207D08B0706D00B78491C0370401C0C
:207BA000521EF7D87047830706D00B78491C0370401C521EF9D1704770B4103A03D378C942
:207BC000103A78C0FBD2530701D318C918C001D508C908C0D20704D30B880380891C801CF9
:207BE000002A01D50B78037070BC704718B40022426001602A490A68002A02D1086011BCA4
:207C000070470A0000E0221D1468002C01D0A042F9D24460106008680028F0D000E008000A
:207C200041680029EBD0026883188B42F7D14B684360096851180160F2E7002018490968C1
:207C400004E00A68904200D2100049680029F8D1002800D00838704718B401000020C91DB5
:207C60000722914308310E4A00E01A1D1368002B14D01C68A14208D218005B18136002682C
:207C8000521A1A6042685A6004E08C42EDD118005B681360002801D00160083012BC7047C5
:207CA0002C0B0020002800D1704780B508380168FFF79CFF01BD80B5CA1D07218A43083245
:207CC000083801680260891A8018FFF78FFF01BD10B504002068FFF7E5FF0020206010BD84
:207CE00080B507229143FFF781FF01BD10B572B6074C6178491C617008220021FEF7D6FBBE
:207D00006078401E60706078002800D162B610BD78010020F0B583B00020694608801424A7
:207D200001F048FA002800D0102401F041FA002801D0382084430122012100A8801C01F026
:207D40007BFA68468078012802D0022806D00BE00422002101A801F005FB15E004220821FD
:207D600001A801F069FA0FE088480190102C0BD101220021684601F05FFA68460078042810
:207D800002D26846012141700198814F3E000B360C2502AA0A21FEF790FB02993031317081
:207DA000761E6D1EF5D1FF20801C69464978002903D06946097808180CE0102C0AD0142C25
:207DC00001D1001D06E0042C01D1401D02E0802040012043788203B0F0BD80B5FEF7DDFFE9
:207DE00001BD10B50C00A007800F022801D0FEF7D4FF600702D567480121017010BD30B5C9
:207E000083B0FFF787FF01F057FC02F0AFFA604C01F0CEF900281FD101AD00900023402295
:207E20000221012001F0B5FB28704020009023002C3340220221002001F0ABFB687001A896
:207E400002F076FB5449002002F0B8FB002253492000203001F0A4FF1034200002F082F9CA
:207E600001F05EFC03B030BD80B501F086F91420FEF70FFD01F080F901BD10B582B00C0012
:207E8000474909680091002322000100002002F0F8FAA04204D0002001F068F901F036F9BE
:207EA00013BD10B582B03E4C20680090012300220021002002F0E5FA2168002002F087FBE4
:207EC00013BD10B50C0036490B6822000100002002F0CCFAA04204D0002001F047F901F01C
:207EE00015F910BD38B505000C002D480168002002F075FB002804D0002001F037F901F01B
:207F000005F90020C0430090002322002900002002F0B7FA002804D5002001F027F901F05C
:207F2000F5F831BD10B50C001D490B6822000100002002F0D0FAA04204D0002001F016F9E7
:207F400001F0E4F8002010BD80B50A000100002002F0CAFA02BD80B5002002F0DFFA02BDB3
:207F600080B5002002F0D2FA02BD80B5002002F0C4FA02BD80B501F054FF8007800F0228B2
:207F800001D1012002BD002002BD000040E201000C010020631B0020DB7D0008E37D00089A
:207FA000080100204020704738B5040072B6104D6878401C687001202071206800280ED0B7
:207FC0002878401C2870200002F034FB002804D16079012801D000202071FEF7B4FB6878C7
:207FE000401E68706878002800D162B631BD00BF7801002070B5040072B60F4E306A45186F
:20800000207900280CD12A004821200002F036FBB068C068281A012801DA012070BD72B6F0
:208020006079012801D0002020717078002800D162B6002070BD00BF78010020F2B584B043
:208040000600356E706E316D88421FD0042204A92800FFF79DFD2D1D002401E06D18641C63
:20806000306B844215DA2001F16A0818029000200190009502988368426801683000F76914
:208080007F68B847029949688842E7D00020C0430BE0B06D316D41188D4200D105003566CB
:2080A000706EF16B40187066002005B0F0BDF8B5070004216846FFF735FF786E002802D144
:2080C000FEF700FEF1BD0098F96B02F011FB0090F96B48430090786E0099884200D90800CC
:2080E000009004216846FEF786FDFC6D009D02F033FB386DB96D0818061BB54200D22E007C
:2081000031002000FEF777FDA419B86D396D41188C4200D10400AD1BEBD102F022FBFEF799
:20812000D7FDFC65786E0099401A7866F1BDF8B504000026009604213030FFF7F3FEE66284
:20814000206B0B2805D20001FFF786FDE06200281BD10120C0430090206B00010830FEF74D
:20816000D3FDE06A002801D0FFF79CFDA06D002801D0FFF797FD3C2200212C342000FEF7D9
:2081800095F90098FEF79EFDF1BD216B0901FFF7C9FE042120003430FFF7C4FE0421200082
:2081A0003830FFF7BFFEE663206B012808DBE16A091DE26B0B68D218E2631031401EF8D1FC
:2081C000E06B001DE063616B642900D26421824A504302F08DFA0500A06D002806D0216DCE
:2081E000A94221D0FFF75EFD2665A665FFF725FDE76B4100081840000A2102F079FA3900E8
:2082000002F076FA7843854200D90500BD4203D32800FFF721FDA065A06D002803D101205C
:20822000C04300909DE725656665A06DE065A06D2066FA25AD003820205CC00709D502F0B6
:20824000BFFA0600606B37183000290002F03CFA07E06248066A606B290002F049FA37184B
:208260003000E0646664276400212000FFF7E6FE87E710B504000120616D01400CD1A16BCA
:20828000084002D002F09CFA01E05448006A616C0818A16C401A606410BD10B50400012086
:2082A000616D014008D1A16B084002D002F088FA01E04A48006AA06410BD8D22825C002AD7
:2082C00000D0704738B5383004002278D007C00F00290FD10125E169294020D1002802D0B1
:2082E00002F06EFA01E03D48006A2061E0690543E56131BD012912D1217FC9070FD5002885
:2083000002D002F05DFA01E03448006AE16808182169401AE060E06901218843E06131BD89
:20832000F0B583B0040001250195206B002850D0E06B00284DD000260196A06B284003D03F
:2083400002F03EFA070001E02448076A206CC01B01283EDA616BA26B2A4007D100900800D3
:20836000FA21890002F0C4F901000098401800D5002038182064194E306AE16C814218D0F7
:20838000E0642069E169096A8847002807D1606D284012D001212000FFF78FFF0DE0012891
:2083A00017D1606D054014D100212000FFF785FF0FE0606D2840C0070BD4A06B054002D037
:2083C00002F0FEF900E0306A616C411A2000FFF735FE019803B0F0BDA08601007801002010
:2083E00010B58AB0040001216846FFF79BFD6846007800281DD0022807D002D3032814D0FC
:2084000027E02000FFF793FE23E02000303000210160C16A026B8A4201D3501A02E0006ABB
:20842000401A8018FEF74EFC13E02000FFF73FFE0FE001900A210291FA21890003910490BB
:2084400005900690079008900990242101A8FEF7C7FB8C34012020700AB010BD18B40200BE
:2084600000230020FF24A41CA24208D07D4CA24205D07D4CA24202D07C4CA24200D17C48D8
:20848000002900D00B6012BC704770B50600FFF7D4FB050080204001854202DAFFF7CDFBBC
:2084A0000500002D25D02800FFF7D6FB04002A0021003000F369DB6A9847002816D4291A52
:2084C0002000FFF7F8FB34610020B0843062F069006800280DD0FFF7B0FB0100F0690068EF
:2084E000814206DBFFF7B8FB306270BD2000FFF7D9FB70BD10B5C100081800015D490C18E8
:20850000206900282DD0206A002803D020002030FFF7DEFBA06D002803D0FFF7C3FB00200D
:20852000A065E06A002803D0FFF7BCFB0020E062606F002803D0FFF7B5FB00206067A06E7D
:20854000002803D0FFF7AEFB0020A0666069002803D020001430FFF7BBFB10342000FFF72D
:20856000B7FB10BDF8B50C00042826DA2168090E0025FF2900D100210E0221790E43C100FC
:20858000091809013B4A5718FFF7B4FFFF20801C864208D03348864205D03348864202D08B
:2085A0003248864200D1324DE561902221003800FFF702FB3800FFF768FFF1BDF7B50700EF
:2085C0000E001D00454CE069C26C100013D0012120699047002001900095029B32003900A5
:2085E0002000E5696D68A847050000212069E269D26C90470AE0002001900095029B32003B
:2086000039002000E4696468A0470500280003B0F0BDF4B582B007000E001D00304CE069A2
:20862000C26C100011D00121206990470095029B320039002000E569AD68A8470500002164
:208640002069E269D26C904708E00095029B320039002000E469A468A0470500280003B06C
:20866000F0BD00000103000001060000010E0000045B0008D012002038B5194CE169CA6CF8
:20868000206913000CD0012190472069E169096A8847050000212069E269D26C904702E063
:2086A000096A88470500280032BD38B50C4CE169CA6C206913000CD0012190472069E16953
:2086C000C9698847050000212069E269D26C904702E0C96988470500280032BDD012002089
:2086E000D0120020010088684A68801A01D5C96840187047010048688A68801A401E01D5B4
:20870000C96840187047F2B504001500FFF7F2FFA84203DA2000FFF7EDFF05002E00A0686E
:20872000E16822685118091A37008E4200DD0F003A000099FFF72CFAA068C0190099C9199C
:208740000091F61B2168E2688A18121A00D10800A060002EE3D12800F2BDF8B504000D0086
:2087600001F0FAFF8F4F381D02F09AF86068E168226851180E1AB54200DA2E00002E03D02C
:208780003100FEF738FAAD1B002D03D029002068FEF731FAAD192000FFF7A4FFA84203DAA2
:2087A0002000FFF79FFF00E02800002810D00500E1682068411862688B1A9D4200DC2B0071
:2087C000D2186260ED1A891A00D16060002DEFD1381D02F085F801F0C4FF2000FFF782FFB6
:2087E000050061682068E2688218521AAA4208DB012D02DB2A0002F08BF8206860604019B9
:20880000A060F1BDF0B583B0050016001C00089B0020019000942800EF697F68B847B0425B
:2088200002D00020C0432AE06879002826D06069FDF7D8FD60612069FDF7D4FD20611834CC
:20884000002618E02068FDF7CDFD20606068FDF7C9FD6060A068FDF7C5FDA060E068FDF7F8
:20886000C1FDE0602069FDF7BDFD20616069FDF7B9FD6061761CE86E8642E3DB002003B0CD
:20888000F0BDF0B583B00400002708216846FEF731FA0198012860DB0025434EA6422ED098
:2088A000B06E00282BD0706F002828D030682168884224D130792179884220D10422210053
:2088C00008313000083002F036F8002817D1E8004019000134490D18686F002802D0FFF71C
:2088E000E1F96F67A86E002802D0FFF7DBF9AF662022002168352800FDF7D8FD03E06D1C7C
:208900009036042DCADB656F002D0CD02800FFF7C9F9A06EFFF7C6F9202200212000683020
:20892000FDF7C4FD0025019841000E18F6003000FFF792F9A06632000021FDF7B7FDA06EA7
:2089400000280CD0FFF779F9052101F0D1FE0600FFF782F9050019D10127FF4306E00127E7
:20896000FF43002D07D02800FFF79CF9A06E002801D0FFF797F92022002168342000FDF75E
:2089800095FD3800FEF79EF903B0F0BD009820670198E066802026506567A567E567843431
:2089A0002770EEE7C80B0020D0120020F1B590B0614E3068002804D101203060301D01F03D
:2089C0005AFF1098743002901098C06E002800D124E102980068002800D11FE11098843035
:2089E0000078002800D019E110980068000E082803D00C2801D00F2801D1022000E00020BC
:208A000000060E900298FFF775FE042849DAFFF714F905900298C0680599884200D3FDE0EE
:208A20000846FFF719F9040000D1B4E1301D01F037FF0298416882688A420AD3521A2000A0
:208A4000FFF7A6F80298806802994968401A201817E0C26803689A18551A2A002000FFF735
:208A600097F8029801688068421A6019FFF790F80298C06802998968029A5268891A611869
:208A800008180299886002994C6002980599C16002980068FFF706F902980460301D01F060
:208AA0001FFF1098C06E41000D18ED0018352800FFF7D2F8040000D199E00E980090230093
:208AC0002A001098016FFFF79DFE00280DD4207853280AD16078452807D1A078472804D153
:208AE0001098C06E2169814203D02000FFF7DAF851E12100183103911099896E0191002214
:208B00000092012843DB002200258E68002E039B14D19B68002B34D0A04DAB4200DBD24392
:208B2000039D2D69AB4201DA0022D243039DED68AB4259DB1EE000BFC80B00205B684F68C0
:208B4000BB4200D0D243039B9B68B34201D00022D243039E3669B34201DA0022D243039EAD
:208B6000F668B34201DA0022D243039B1B680E68B34200D00125002A35D1002D01D00122BD
:208B800000921831039A18320392401EBBD1206941000A18D200210018310198FEF7F8FFE7
:208BA0002000FFF77FF8009800282DD0206941000C18E4006846FF210174029806A96CC8D9
:208BC0006CC106A8FFF796FD844204A811DA4470200A04A98870032206A8FFF794FD2200D5
:208BE0001098816E0AE0CAD52000FFF75BF80020CFE0002141708170032204A906A8FFF7E4
:208C000082FD0298089981601098806E039000270298FFF76FFD0400042C01DA0120B8E0A5
:208C2000039840680A900399096941180B91039AD26880180C90039880680D900398183046
:208C400003900D98002800D19CE00F919748844200DB441EE41E0AA8FFF744FDA04203DA3B
:208C60000AA8FFF73FFD0400002C00D593E000D188E0029806A96CC86CC16846077404A8E0
:208C80004470201204A98870032206A8FFF73BFD08980999069A5118091A25008C4200DD0A
:208CA0000D000B990D9A0A9B9A18521A954200DB15000022019200900E9B2A001098C669E3
:208CC0007668B0470600AE4265D106A8FFF712FDA84203DA06A8FFF70DFD00E028000999C1
:208CE000069A5118089BCA1A904200DC02009B180893801AC91A01D1069908910028EED178
:208D00000AA8FFF7EFFCA84203DA0AA8FFF7EAFC00E02800002810D00D990A9A51180B9B02
:208D2000CA1A904200DC02009B180B93801AC91A01D10A990B910028EED1641BA8D1002EB3
:208D400029D40298089981600B980F99884219D07900C919C900109A126F8C1828340A990A
:208D6000401A059010984079002802D005A8FDF72BFB05A800900E9B042221001098C469E0
:208D8000A468A04700207F1C1099C96E8F4200DA3EE711B0F0BD0020C043FAE70100000101
:208DA00070B584B0040042480168002904D101210160001D01F05FFD012102A8FFF7B2F80C
:208DC0006846007A05280CD801A1095C8F4400BF061C24347A8E0320009004216846FDF7C5
:208DE000FFFE8C340120207004B070BD2000FFF748FDF6E720006C30012101760020FDF783
:208E000061FFEEE70025042101A8FFF78BF8260074363068002806D0E06E002803D03000D2
:208E2000FFF760FC05002800FDF7F8FE002D09D00198002806D00146A94200DD29003000C4
:208E4000FFF78BFCFDF744FFCBE72100743100200A68002AD3D00800FFF744FCCFE704216E
:208E60006846FFF75FF8250074352868002815D0E06E002812D02800FFF734FC0099002924
:208E8000E0D000280DD00E46864200DD060031002800FFF762FC0098801B009000980028EE
:208EA000D0D0FE210098FDF7BFFECBE703000100C80B002008B4024B9C4608BC6047C046A5
:208EC000ED050020F8B408B40D000799032443009C40E3439024E40526681E402660266862
:208EE0004700BD403543256001258540A6882F00BE43A6806E463678002E02D0A6883743B8
:208F0000A780A6681E40A660A668B4466E46377E4600B74066463743A760E6683340E360D9
:208F2000E368400082401A43E260002903D0A0690543A56102E0208D05432585F3BC70470B
:208F400055480168802292020A4302609020C005A02189050160C168524A0A43C2600121AB
:208F60008161026803239A434AE04F4870474F480188C806C00F70474C4801884807C00F7B
:208F8000704700207047494800880107C80F7047464801888807C00F704701207047FF2071
:208FA00070479020C00501683022914301600168684A0A4002600CE09020C00502210185C4
:208FC00001680C22914304222CE09020C0050221816101680C229143016070477047704789
:208FE000704770479020C0051021018503E09020C005102181610168564A0A40802149002F
:20900000114301607047704770479020C0050421018503E09020C00504218161016830223C
:20902000914310220A430260704780B5FFF7EDFFFFF7F0FF01BD52484068704710B501004B
:209040004F4C616010D0002020603848007801280AD14C4A914204D24B4801F049FB001F12
:2090600001E00020C043206010BD10B582B0040008004349096800912100FEF711FC0020CB
:2090800016BD2A490978012901D8182100E0302181803E49016070471410024070473C485B
:2090A0007047000055555541E40C000010000048012800D0704700B583B000200190032005
:2090C00000900023002201210220FFF7FBFE01200190032000900023012200210420FFF7A2
:2090E000F1FE0120019003200090002301220021FFF7E8FE0120019003200090002301222E
:2091000000210120FFF7DEFE03B000BD72B601F035FC2048022101601F48FFF7CBFE1F4808
:20912000016889B21E4A0A430260FEE7611B0020002806D0401E032806D90938022803D946
:2091400004E0094800787047002070470020C04370470000FFFCFFFF7047002802D11148F6
:209160000121018070470000581B0020002802D10D48012101607047704770470B48704700
:20918000EC0A002080841E00808D5B00006CDC02102700004060004020A107000CED00E02D
:2091A0000700FA052800004818000048FF3F00200020704780B501228921684600F03CF8D0
:2091C00068460078012803D068460078FF2801D1002002BD012002BD0120C0437047FEE7CF
:2091E00008B4024B9C4608BC6047C0461705002008B4024B9C4608BC6047C04697030020C1
:2092000080B57348002101600120FDF74FFD6420FDF73FFB72B66F484178491C41706A4869
:209220006A490160FFF772FF01BD6B480178002901D16A4810307047F0B506000C00150059
:20924000002E1ED0002D1CD060196549884218D2C80884420FD2001B2F00854200D9070096
:209260003A00604821183000FEF792FCF619ED1BE419002D05D02A005A4821183000FEF7E0
:2092800087FCF0BD80B55748FFF7AAFF002002BDF0B5C1B00C00150000280AD0002D47D0CF
:2092A000070080200001844203D260194C49884202D30020C0433CE0FF2C1ED8802040007E
:2092C000061B864200D90600AE4200D92E00320039006846FEF75CFC0023320069464148DC
:2092E0002018FFF785FFBF19AD1BA419FF2C02D8002DE3D11CE0002D1AD0FF20C043241808
:20930000FF20801C854201D3461E00E02E00320039006846FEF73CFC0023320069463248C1
:209320002018FFF765FFBF19AD1BA419002DE7D1002041B0F0BD38B5040007D0002901D1D8
:20934000002032BD80252D01A94202D00020C04332BD2448FFF744FF2A0000212000FFF756
:2093600097FF32BD002800D1704710B5002A0FD08B18FF24A41CA3420AD2631E994207D26E
:209380005B1A9A4200D91A00184BC918FEF700FC10BD10B5C0B080246400A14201D100286D
:2093A00002D10020C0430BE0220001006846FEF7EFFB0023220069460C48FFF719FF0020A6
:2093C00040B010BD0000000000010020214334124812002078010020BC11002000490008B4
:2093E000010800000040000800410008003F0008F9B583B00D0017000101081A8000AC49EE
:209400000E18AC4C2000A430009080698047B079012801D1022496E0E41D0294E0788007C4
:20942000800F022800D08DE0306900280FD1707EC107C90F684601710A980A90002D45D168
:20944000002F43D1002843D1706A002801D0032479E00024012500212D193A1B0020029B77
:209460001B78002B06D0049B002B02D10A9B002B00D0012072613561B176F07600990988DA
:20948000491C009B19803181317E00290DD13188914202D2002800D00A0029000398009B0A
:2094A0001B69DB6A9847012030760A9802284BDA049800283BD00146039801F083FA002805
:2094C00038D00021039800F01BFE33E0002F02D16846012101713A00290030001C3000F099
:2094E00035F90400381B04D00A98012815D1002C17D068460079002826D0306A716A401A3B
:209500003188884220D302200A90002168460079002819D000220025A0E7002102289BD13B
:20952000F4E701213088B84296D2070094E7039801F041FA70693C1A0298C0788007800FB4
:20954000022801D00024E4430098C0698047200005B0F0BD18B401002031447F641E012C2B
:2095600005DB0A0008320CCA0CC1641EF9D1417F491E417711BC704738B50C00856B04E0A8
:20958000A96820006A6890472D68002DF8D131BD7047FEB582B007004648B430006800906B
:2095A000002644480078062853D2694608710101081A80003E490D180098C36C0A980A90B3
:2095C000180005D00A9A6846017A3800984705E06846017A3800009A52689047040038D03D
:2095E000FF2C36D03C212800FEF720FAF901214369716846007A287168460079009949693B
:2096000088470600002F03D10A98B04200D8060000F0FEFCC2B26846017A300000F0C1FC9C
:209620002880684680896880002F03D02048C068E86003E00498E8610A9828621D48007838
:209640000600401C1B4908706000C0190818F8300670300005B0F0BD410601D10020704753
:209660000107C90E000600D5491C9F484018F830007870470101081A80000D490818407962
:2096800070479948817A8807C00F7047F8B5094FB4203C580125064E03E03000A168884750
:2096A0006D1C3C3638788542F7DBE0688047F1BD040E00206C0F0020F8B50020C04300907C
:2096C000894C8E2149002000FEF7B0F901272770A72032212154B94DB42149002800FEF770
:2096E000A5F901F057F901F0BDF9B42026582000EC300168002901D1B1490160706D0100B9
:2097000000D080470020716988472880326C100002D06946052090470098E8606772F1BDAF
:2097200038B5714CB4202558286880472A6C100007D0E11D062090472100083102202A6C4D
:2097400090471020A0722869804731BDF2B504001500002621E0002924D0E068411862683B
:209760008A4200D90A00171AAF4200D92F003A00216809180098FEF70BFAED1BA068C01BAF
:20978000A060F6190098C0190090E068C019E0606168884201D10020E060A168002DDAD1B2
:2097A000002901D10020E0603000F2BDF2B5040015006068A168461A1CE0E068A1684018D9
:2097C0006168884200D3401A4219914200D911000F1AAF4200D92F003A0000992368181801
:2097E000FEF7D6F9ED1BA068C019A0600098C0190090F61B002DE0D13000F2BD10B500F038
:20980000B5FC80B500F0B8FC10B582B0002B02D50224002300E0012400F0AAFC80B5674BFA
:2098200018625962012058779A76002018832E49B4310968096B884701BDF7B504001F009B
:20984000294EB07A8007800F022801D0002008E02001001B800059490D18A879002802D0B0
:209860000220C0433DE0A436B0698047687F00281FD0C100691818314A680B689B18019CEE
:20988000A34204D1029810184860AF7625E0032802D10324E44321E008310C600298486046
:2098A000687F401C6877AF763088401C3080288113E0290020310198086002984860012023
:2098C0006877AF763088401C308028812869002803D120003169096B88470024F069804749
:2098E000200003B0F0BD00006C0F0020F2B582B004002001001B800030490E18824D28001E
:20990000BC300190006800277179090631D50097002580473069002802D1707F002820D01E
:2099200037770298002819D00146200001F04AF8002816D03069022800DB451E30002030A5
:20994000717F012905DB4268AD180830491E0129F9DA0021200000F0D3FB02E0200001F010
:209960002AF8019840688047002D23D00120009020E080473069002818D0029800280BD0DF
:209980000146200001F01EF8002808D00021200000F0B6FB012702E0200001F00CF8A87A36
:2099A0008007800F022801D00027FF430198406880470097009803B0F0BD0000040E002064
:2099C00091950008F8B504000F002001001B80004E490D1800264C48BC30009000688047BC
:2099E000687F032814D3002F01D5012610E001202877002F07D03900200000F0E3FF002839
:209A000004D0012602E0200000F0D5FF002028770098406880473000F2BDFEB504000F001A
:209A20001500089E002E02D5FFF707FF4EE06846037A2A0039002000FFF7FFFE0321C9436B
:209A4000884206D131002000FFF7BCFF0028EED03BE000283AD4019600272001001B8000B2
:209A60002A490E182848BC300090006880473069002802D1707F002820D037770198002828
:209A800019D00146200000F09DFF002816D03069022800DB471E30002030717F012905DB5F
:209AA0004268BF180830491E0129F9DA0021200000F026FB02E0200000F07DFF0098406889
:209AC0008047AF4201D2E81B00E0002003B0F0BD42001018C0000C4A101801637047420093
:209AE0001018C000084A10184163704706490A00A6321378032B06D29B00C918A83108602A
:209B00001078401C107070476C0F0020040E0020F2B582B0060015003001801B8000AC4928
:209B20000C18002E12D10024B14E3700A6373878844261DAA0003018A8300268100002D0FC
:209B4000290002989047641CE4B2F0E7E068002803D029000298E26890470120009020691D
:209B600000282CD061698D4201D22F0000E06769002F0DD03A000299FEF70AF8ED1B0298FC
:209B8000C01902902069C01920616069C01B60616069002802D0A07E002810D0300000F009
:209BA00003FF00272761607EC00706D430009049B4310968896A8847277609200090002DD1
:209BC00016D02A00029920001C30FFF7EFFD617EC90702D5218888420AD2207E002807D01A
:209BE00030008349B4310968896A88470020207600992000FFF7C0FC03B0F0BDF8B506001D
:209C00003001801B800072490D18687F002874D0002E02D0296900296FD10021E9762F001B
:209C200020377968002904D1022802D32800FFF791FC6F48B43003681C6D20001AD0288BF8
:209C400000906B463A00697F3000A047040000982883601C2861260003E0361A2800FFF7C7
:209C600079FC7868B042F8D3801B78603868801938601FE07C682888844200D90400601CDC
:209C800028612200396830005B6B98477868001B7860386800193860002C03D02988481E69
:209CA000204001D0002010E02E8B200000F020FD301828836869002808D0298B002905D007
:209CC0002A885143401E084000D128837868002813D1687F022803D32800FFF73BFCF1BD46
:209CE000002C08D0288B002805D0A87E002802D00020A876F1BD00206877F1BD38B5040006
:209D00002001001B800032490D18002C0DD0286902280ADB0020C04328610421E87E0028DF
:209D200000D106212800FFF727FC00202861687F00280CD02000FFF761FF687F032818D2E4
:209D4000287F002815D0200000F02EFE31BD20002749B4310968896B8847002C07D0200059
:209D600000F022FE40212800FFF706FC31BD01F09CF931BD80B50201121A9200144B9A18E9
:209D800091711B4AB4321268126A904701BD80B50121FFF7EFFF01BD1549B4310860704790
:209DA00038B400230024002538C00C3841608260A6490A68130000E01B68002B03D08342F2
:209DC000FAD1012002E002600860002032BC7047040E002010B40401201A80009C4C201851
:209DE0004A608B60826B0A60816310BC704700006C0F002010B59748817A0021017301221E
:209E0000934B423302E01970521C3C330478A242F9DB817A102001400820084300F014F898
:209E200010BD8C48807A704780B58A48817A0120084300F009F801BD80B58648817AFE2097
:209E4000084000F001F801BDF0B583B00700814EB47AB42030580190BC4249D0A00719D49F
:209E6000B80717D5012568460570FFF70FFC07E000212800FFF77EFF280001F059FA6D1C55
:209E800030788542F4D30198026C100002D0694600209047A0070BD5B80709D4684600210B
:209EA00001700198026C100002D06946002090478C204000345806E06268100002D039005F
:209EC000A06890472468002CF6D1B772B07A062108420DD0012408E00021200000F010F93C
:209EE000200000F0B9F8641CE4B230788442F3DB03B0F0BD01000020564A927A9207920FE8
:209F0000022A05D10801401A800051490818406A704738B505004F4CBC342068804728014C
:209F2000401B80004A4908180169022901DB4D1E00E0002501002031407F012805DB4A68E6
:209F4000AD180831401E0128F9DA60688047280032BD0101081A80003D4908184069704759
:209F60000101081A80003A490818417F002902D00020C0437047018B4269002A0AD00029A1
:209F800006D003885943521E0A4008D10021018300207047481E8041C043C00F70470120E4
:209FA00070470200032905D14020824213D24008FBD17047402A01D340207047202A01D39F
:209FC00020207047102A01D310207047082A01D3082070470020704701700A0A42700A0C8C
:209FE0008270090EC17070470170090A417070470178427812020A43817809041143C0785E
:20A000000006084370470178407800020843704780B52848B43000688069804702210840F7
:20A0200002BD80B52348B430006880698047C007C00F02BD1F4A5078411C517041000918BF
:20A04000C90051182A3108707047000084100020040E00206C0F002070B504002001001B5E
:20A06000800048490D180026AE716879000604D52E616E772E8320210DE06E62AE622E61E3
:20A08000287E002805D020003F49B4310968896A88472E7610212800FFF76EFA200000F0F2
:20A0A00083FC70BD0201101A8000364A1018C160704700006C0F002078B4010001200024BA
:20A0C000314B1D00C826AE59002E05D1A0001818C8300160002003E0641C2D1D052CF1D303
:20A0E00072BC70472849DC31086070470201101A8000244A10184279120600D44176704786
:20A10000F8B504000F002048B43001682001001B80001C4A1518002C19D000266879000659
:20A1200007D52000896B88472E616E772E83202105E02000896A88472E762E6110212800A7
:20A14000FFF71AFA002F02D0200000F02DFCF1BD0D49EC31086070470B4BB8331860596009
:20A160009A6070470849F4310860704782B000240094FFF73DF916BD032300930023FFF7DE
:20A1800037F902BD040E00206C0F002010B59E4CE168002904D1006801F0A0F90120206179
:20A1A00010BD7047800700D1704780B500F0DEFA01BDF0B589B0FFF734FE8007800F02280B
:20A1C0000CD1914C2068002808D060688F49096A401A012802DA2069002801D1012046E001
:20A1E00001256069002804D12000183001F07AFA6061616900290ED00023DB43A269A068C0
:20A2000001F095FB002806D4E069A1694018E061002666610025E069002809D0A06801F07A
:20A2200095FB0500E069401B01F04EFAE56101E0002D00D10027012504E000250100684682
:20A2400001F09FF901F037FA202802DA002801D109E020200023DB4302006946A06801F021
:20A260005CFB0128E9DA002D00D10027380009B0F0BDF0B585B000250027012101A8FDF7F3
:20A2800051FE04216846FDF74DFEFEF793FF0028009804D0FCF738FD02AC5D4D51E0083059
:20A2A000FDF7DAFC040005D10098FCF72DFD02AC012545E00099FDF735FE6846007900283D
:20A2C00006D0022829D00CD3042832D02BD336E02000FCF7CEF80100201D01F052F905000C
:20A2E0002FE02000FCF7C5F806002000FDF7DAFC30000830FDF7B0FC040002D102AC0125DC
:20A300001EE03100083001F07BF907003E483F49096AC2688918416013E02000FCF7A9F8D6
:20A3200001F028F90DE02000FCF7A3F83649C86007E02000FCF79DF801F0D0F801E0022579
:20A34000ED4329002000FCF77FF83900201DFCF77BF8083739002000FCF742FC02A8844205
:20A3600002D02000FDF79EFC05B0F0BD7CB5264CFEF720FF012141402160FEF719FF0028EB
:20A3800004D1206800283BD001F0F0FB2068002836D001AD40200090002300220221012074
:20A3A000FFF7F7F828704020009023002033002202210020FFF7EDF86870002000900023CF
:20A3C000082203210120FFF7E4F8A87001A801F0C9FAA0600F4901F092FA0F49A06801F0A1
:20A3E00095FA0E4E00233200210060316878FFF7F1FC0023320021006C312878FFF7EAFC19
:20A400000020E06073BD0000540A002078010020FAFEFFFF8DA10008A3A10008A5A10008CF
:20A4200080B50178412917D14178012914D1C1780902807808438021C901884201D2800243
:20A4400001E0400A400200F0D6F8012200210020FFF7E4F9002002BD012002BD480700D5B7
:20A46000704780B5002000F0C6F801BD10B582B00093012344002018644C205CFFF7CDFA51
:20A4800016BDFBB517004100081860490C5C089E002F16D12000FFF763FD0500012D10DA61
:20A4A000002E04D5002D14D00320C04311E031002000FFF71BFA002801D1002DEAD100200F
:20A4C00007E000966846037A3A0001992000FFF7A4FA03B0F0BD10B5440020184B4C2018DC
:20A4E0004078FFF78BF910BD80B543001818474B18184078FFF785F902BD80B54100081872
:20A50000424908184078FFF7F5FC02BD80B5410008183E49085CFFF7FCFC02BD80B541008E
:20A5200008183A4908184078FFF713FD02BD0000F1B50126354C2079002804D1267160718F
:20A540003348FFF7B9FDFFF775FD050068004019C00030490F182437FF20F87038717871D2
:20A5600000980078012181400098407886400E433E8000BF2BA000F0E5FEF87160794100E3
:20A58000081820180099097801700099497841708570214E31002800FFF7A1FA002D03D07F
:20A5A00031000020FFF79BFA00221C4920000830FFF7F6FB6079411C6171F2BD80B54200CB
:20A5C0001018124A10184078FFF76CFD01BD80B5420010180D4A105CFFF788F902BD80B52D
:20A5E00042001018094A105CFFF7ECF902BD0748002101717047054909780A01511A890031
:20A60000074A51184861704700000000200C0020EFA500086C0F002021A400085DA40008C7
:20A62000040E002042554C4B20696E746572666163650000F8B50700002472B60E4D6878AE
:20A64000401C687004260BE0C068017C314205D0C1682A6A891A012900DA0124FCF78CF8C4
:20A6600038680028F0D16878401E68706878002800D162B62000F2BD7801002030B585B0C8
:20A68000029001900F4B9C68039472B69C68E2601D6A521B012A04DA5878002810D162B646
:20A6A0000EE0026800926A4602600098002800D042606846A060042008432074FCF7C6F80A
:20A6C00005B030BD78010020CA0F00D0494203105A400DD004B500D3404200F009F8009AE8
:20A6E000D20701D34942124200D5404204BD0000094210D088420BD30122002300185B41E9
:20A700008B4200D35B1A5241F8D319001000704701000020704708B501F046FA08BDFEE776
:20A72000234D0126280000F0BBF8FDF727F8002800D10026FFF73DFD002800D1002600F046
:20A7400089FF280000F0CCF8002EEAD0012128001030FDF74FFCE4E780B5154800F0C0F8DF
:20A7600001BD80B5124800F09BF801BD80B510481030FDF719FC01BD10B584B00C4C200046
:20A7800000F079F802212000103001F00FFA0220029040020190200018300090054B0122E9
:20A7A00005A18320C000201801F018FA04B010BDF805002021A7000842475461736B0000CB
:20A7C000F8B572B61B482830C0C81948C068804704000025164800698047002806D000203C
:20A7E000761C47411248C06880470400104842690023007A002804D10021101BA94104001B
:20A800000D003000390001F021FA00196941084A9269002301F01AFA054AD269002301F0E0
:20A820002EFA044A5278002A00D162B6F2BD0000580B002078010020F8B507003048046862
:20A84000304D012614E0207A002810D06068B8420DD126722878401C2870207A401E207268
:20A86000000602D1200001F03FFAFBF76CFFE468002CE8D1F1BD10B5040023482349016078
:20A88000102200212000FBF711FE72B61C480168E16004601B484078002800D162B610BDB1
:20A8A00038B50400174D2878401C2870A868217A002902D1606001250DE06168814208D0D1
:20A8C0001021200001F022FA207A0028F8D1A8686060257A6D1C2572FBF735FF280032BDC3
:20A8E00080B508490A78521C0A70017A491E0172090601D101F0F8F9FBF725FF01BD00007C
:20A90000480B002078010020500B002039A8000812420FD0814202D25318984203D310B51D
:20A92000FDF736F908BD80185B1E1978401E0170521EF9D1704718B402E0401C491C521EEE
:20A94000002A09D00B7804789C42F6D002D20020C04302E0012000E0002012BC7047FEE7ED
:20A9600000B58022520009495005FDF725F90848016803220A430260002000BD0448016856
:20A98000032291430160002070470000004800080000014038B5174C06252000FDF7A6F9C7
:20A9A00008346D1EF9D131BD80B5C0001149081801F0C6F901BD80B5C0000E49081801F0DE
:20A9C000DBF901BD80B5491CC0000A4A1018FDF711FB02BD08484178491E4170407800284F
:20A9E00000D162B6704772B603484178491C41707047000088100020780100203548016887
:20AA0000802292020A43026033480168334A0A4002600168BB2212030A4302603048016859
:20AA2000C20B0A43026070472D4801682D4A0A400260704730B42C490860802000062B4950
:20AA40002B4A13680B40034313601368C0242406156829401B191C400C431460254908606A
:20AA600030BC704780B524480168244A0A400260C168802212040A43C26019480168194A92
:20AA80000A4002601E48FFF787F91E4A1E491F48FFF762FB1E48FFF75BFB1E48FFF722FB7A
:20AAA00001BD10B51C4C2078401C20700E480068010000D0804772B62078012804D160684B
:20AAC000002801D0FDF735F82078401E207062B610BD00001410024004080140FF0FF0FF41
:20AAE000585C0040FF7FFFFF980C0020FFFFFF001CE400E000E100E010100240FFFF7FFFA6
:20AB000084F30008D5A90008E7A9000835AA0008FDA9000829AA000878010020026843687A
:20AB20009A4204D2836899540168491C0160704738B504000D00C9B2FFF7F0FF290A2000F4
:20AB4000FFF7ECFF31BD000030B583B0002812D100909F48029080204000019004216846B6
:20AB6000FFF7DCFF03216846FFF7D8FF99496846FFF7DEFF50E0012812D016D3032805D0DE
:20AB800009D3042811D100BF25A51FE09248E0304069C5681AE09048E0304069856815E016
:20ABA0008D48E0304069456810E08B49052807D3401F8A7B904203D280000818056905E091
:20ABC000E03109680A0003D088470500002D01D1002022E028000021002401E0401C641CF7
:20ABE0000278002AFAD10091794802908020400001906100891CC9B26846FFF78FFF0321BA
:20AC00006846FFF78BFF002C06D029786846FFF78FFF6D1C641EF8D16D4803B030BD000008
:20AC2000436F6E66696775726174696F6E00000080B5012200210020FEF7F0FD01BD38B596
:20AC40006549B4228C588278C3781B02134347D18279C3791B021343022B41D1491C032358
:20AC60004A7A520707D40078184239D10B7B5848037002221DE002224D7A154205780FD1A7
:20AC80002B4013D0022B04D03CD20079002827D102E00079002823D14D48002202802EE000
:20ACA0002B4003D0022B16D009D324E00B7B48480370897A11421ED01A4302701BE009784B
:20ACC000491E0079814202DA606A804713E04048002101700FE00079FEF7BEFCFF2802D146
:20ACE000606A804731BD0101081A80008E49081880793749087036480021417000220221B4
:20AD0000FEF78CFD31BDF8B502000C003248B43005689078D17809020143E6B21079032954
:20AD200052DA9379D7793F021F434DD12A4B0A33012909D1002C587802D00221014301E0FE
:20AD4000FD21014059703CE01F787F073CD503271B789B07127814D4174002D0022F03D083
:20AD600032E0022930D12CE000292DD1FEF774FC002829D1601E8041C043C00F6A4988711E
:20AD80001FE0174002D0022F03D01DE000291BD117E0002818D0802816D0FEF75DFC04008E
:20ADA000FF2C11D03100FEF7E5FF002E09D1200000F0BEFA00212000FFF7A2F92000FFF7C5
:20ADC0004BF9FFF735FFF1BD686A8047F1BD0000B8100020090400006C0F0020F4B582B0A5
:20ADE00005000E00108840080024002803E0C10700D5641C4008FAD109212800FFF78EFE2D
:20AE000004212800FFF78AFEF1B22800FFF786FE029881782800FFF781FEE1B22800FFF741
:20AE20007DFE0298C1782800FFF778FE029801792800FFF773FE029841792800FFF76EFEAF
:20AE40000298C1792800FFF769FE02988268100002D02900300090470124334F4037A148FC
:20AE6000B430009006E00126F1B22800FFF756FE641C3C379B480078844253DA02980088D9
:20AE80000121A1400842F3D007212800FFF746FE05212800FFF742FE79782800FFF73EFE49
:20AEA00039782800FFF73AFE3E1FFFF7BAF8002803D100223978308807E0E0B2009909687C
:20AEC000496988470122397880B2FFF76AF8308031882800FFF72CFE2001001B80001249CB
:20AEE00008180179012902D0032906D0BBE74688112E15DA002EB7D1B5E74688FFF791F87D
:20AF0000002807D1FF2E01DDFF26ADE7002EABD10826A9E7112E03DA002EA5D10426A3E791
:20AF20001026A1E703B0F0BD040E0020F0B585B080246C48401C0090807AC00700D5A02449
:20AF40000098007B002802D02000402404430020019065480390802040000290092101A8E3
:20AF6000FFF7DCFD022101A8FFF7D8FD002101A8FFF7DEFD0098017801A8FFF7CFFD012132
:20AF800001A8FFF7CBFD042101A8FFF7C7FD210001A8FFF7C3FD5348A730017801A8FFF7B8
:20AFA000BDFD00254F4F11E06C20305CA84205D132007032290001A8FFF710FF641C1C36CE
:20AFC000009840788442EFDB6D1C183700980078854211DA4348C4300268002A03D001A967
:20AFE0002800526890473A002432290001A8FFF7F5FE00243B4EE3E701993B48801CFEF728
:20B00000F3FF394805B0F0BDF0B583B000200090354F029780267600019612216846FFF72C
:20B020007DFD01216846FFF779FD71006846FFF77FFD2C4C251D29786846FFF76FFD69787D
:20B040006846FFF76BFDA9786846FFF767FDB7480188C9B26846FFF761FDE434206901888C
:20B060006846FFF765FD206941886846FFF760FD2068010002D08047010000E03100684695
:20B08000FFF756FD01216846FFF748FD02216846FFF744FD03216846FFF740FD012168467F
:20B0A000FFF73CFD380003B0F0BD38B50D490C000A34A078000613D5A0784006400EA0707A
:20B0C000A5782800B4310968C9698847002D217802D00420084301E0FB200840FEF7B4FEE2
:20B0E00031BD00006C0F0020B8100020F0B583B0050000269A4C27000BE0380024304169AE
:20B10000080004D028008847002800D10BE1761C1837607802009642EFD32100B43101918A
:20B1200009680E002B7860271F4006D0202F00D1D8E0402F00D1E5E0F3E06A780B2A00D991
:20B14000EFE002A39B5C5B009F4400BF060AEB0CEB1130EB6870859C2800FFF770FDE2E023
:20B16000002100E001212800FFF7CDFDDBE0AD78207A002814D02800C9698847002DA17ACD
:20B1800002D00420084301E0FB200840FEF75CFE2573207A012800D0C5E0FFF749FDC2E02D
:20B1A000FFF746FD802028432073BCE000260024E8790002AF790743684601210170E8785C
:20B1C000012810D012D3032801D004D30EE0A878FFF7BAFC09E0FFF7A9FE0400801CFEF7D9
:20B1E00012FF060002E0FFF70FFF0400002C03D101980068406A95E0002E00D12678BE4291
:20B2000000D93E00BE4202D16846002101706846027831002000FEF701FB84E0FEF731FA16
:20B220006946087000220121684626E0A878012805D1FFF7FDFCA17A0220084306E000284B
:20B2400007D1FFF7F5FCA17AFD200840FEF7FCFD69E0486A66E0A878002811D1A87901280C
:20B260000ED1A07A06220240062A01D0486A59E068460021017000220121FEF7CFFA52E00B
:20B28000486A4FE02A790192A27A06231340062B26D1019A904223DBA878EA781702074387
:20B2A0008020400087421BD2FFF7C2FC01250BE0EEB200213000FEF75DFD300000F038F8A3
:20B2C0003000FEF7C9FE6D1C20788542F0DBF0342268100027D039000198C0B2904722E0FD
:20B2E000486A1FE0287990421BD241000818C00020182430C168080013D02800884700285D
:20B300000FD110E0287990420BD241000818C000201824300169080003D0280088470028FC
:20B3200001D0706A804703B0F0BD0000040E00200B49B4310968C96B0A0000D1704780B564
:20B34000884701BD064A937B052B01D300207047591C91739900511808615B1DD8B270478A
:20B360006C0F0020F3B504006668A068801B01D5216940180090904200DB009200980028CE
:20B380001DD00546206921680818801B2F00854200DD07003A0031000198FCF7F9FB01984A
:20B3A000C0190190F619ED1B2068216941188E4200D10600002DE5D16660E6600098F6BDC0
:20B3C000F3B504001500A6686068801B401E01D5216940180090A84200DB00952069216829
:20B3E0000818801B2F00854200DD07003A0001993000FCF7CDFBF6190198C0190190ED1BDF
:20B400002068216941188E4200D10600002DE5D1A6600098F6BD10B582B08D4C6078002816
:20B4200017D02079A179014313D10020206360630122694620001C30FFF794FF012808D11B
:20B44000A748006A2063012020716846007800F0D8FC13BD38B505007D4CA148006A206313
:20B460006078002803D000F099FD002809D10122290020001C30FFF775FF002801D0002036
:20B4800032BD00202071012032BD10B57049944A126A4A630B69CA68D21A521E01D58C69AA
:20B4A0001219002A0BD018700869401C8B68FF24A41C1C19A04200D118000861521E487898
:20B4C00000280AD0C878002807D1022A05DA086C002802D1012000F051FD10BD70B505005A
:20B4E0005B4C2078002818D100F038FDA0700020E070FF26B61C3000FCF7AEFBA060E06054
:20B5000020616061A6618120FCF7A6FBE061206260628120E06201202070E069002813D040
:20B52000A068002810D0E06B85420AD0A06B002801D0401EA0637A4B7A4A7B49280000F045
:20B5400070FCA06B401CA063002020636063A078607001206071E56370BD10B5734CA06BD1
:20B56000002806D0401EA06303D100F0D9FC0020E06310BD72B66D490122CA70086462B6E4
:20B580007047F8B5324CA26B002A36D00A00010020001C30FFF714FF0500012D2EDB0127A8
:20B5A000A77100262079002823D16079002807D0667100F0F3FC01281DD1667000F0E7FC4A
:20B5C0006078002803D000F0E9FC002811D1266366630122694620001C30FFF7C3FE012849
:20B5E00007D13F48006A206327716846007800F008FCA67102E06770E5E700252800F2BDB5
:20B6000038B54A4CA26B002A1DD06269E3689A4201D0002032BD0A00010020000830FFF758
:20B62000A1FE0500607800280ED0E07800280BD1002D09D0206C002806D0002000F09EFCF2
:20B640000020206400E00025280032BD00000000DC0B002070B582B00126344CA6710025E9
:20B660002079002823D16079002807D0657100F095FC01281DD1657000F089FC6078002885
:20B6800003D000F08BFC002811D1256365630122694620001C30FFF765FE012807D1104816
:20B6A000006A206326716846007800F0AAFBA57173BD6670E5E71D49086A4A6A801A401EDF
:20B6C00001D5C96A401870471849CA6810188A698B689B18984201D35342C018C860704704
:20B6E0007801002078B40100104A53691069984202D2906995682818C41A0AD018001B190D
:20B70000956996687619B34201D36E429B19536100E00020002900D00C6072BC7047000073
:20B7200017B400088BB4000855B40008DC0B002070B50400844D286E002820D442001018C1
:20B7400000012E18072903D00020FEF720FB0EE02000FEF74DFC706020793072607970725D
:20B76000A079B072F168080001D0301D88470020C0432866012200210020FEF74FF870BDC2
:20B7800038B5027941790902114300236E4A1400143401E05B1C3034714D2D78AB4248DAC3
:20B7A00025888D42F6D1002B43D45900C918090154184178202906D03BD3222918D004D364
:20B7C000232926D035E0136631E0251D296820002630FEF701FC20002A30297901706979DE
:20B7E0004170A979817000220721263420001CE0241DE168002915D069468278D307DB0FC0
:20B800000B7080788207D20F4A706846E168884708E0241DE1690A0004D0C2781202807834
:20B8200010438847012200210020FDF7F7FF002032BD012032BD70B50C00002242490B0090
:20B840001433474D2D7801E0521C3033AA4203DA1E888642F8D101E00022D24350008018B6
:20B8600000010D1805212000FFF758F924212000FFF754F900212000FFF750F988214900FB
:20B880002000FFF755F905212000FFF747F924212000FFF743F901212000FFF73FF903219D
:20B8A0002000FFF73BF9A98CC9B22000FFF736F904212000FFF732F924212000FFF72EF961
:20B8C00002212000FFF72AF906212000FFF726F905212000FFF722F924212000FFF71EF9E7
:20B8E00006212000FFF71AF9A98AC9B22000FFF715F9A98CC9B22000FFF710F970BD4200E8
:20B9000010180001624A1018C16070474200101800015F4A10180161704710B544002018BC
:20B9200000015B4C20184078FDF76EFF10BD10B582B000930123440020180001544C205CFA
:20B94000FEF76BF816BD0000340C002080B54100081800014E49085CFEF7DBFA02BD000041
:20B960005D1B0020F1B582B001244A48407800280FD148484470464D60212800FCF756F81F
:20B980004448002101700020C04328664248FEF793FB4248FEF7AAF8FEF74CFB05000195D3
:20B9A0003F49FEF795F868004019C0003D490D1824353D48A8600227EF702F716C710298CC
:20B9C000807801218140298038A0FFF7BBFCE871FEF730FB050068004019C00031490E18BF
:20B9E00024360020B0600A20F07000203071707102980078012181400298407884400C4337
:20BA0000348000BF2AA0FFF79DFCF0712548C4300468002C09D0002000900223022202210B
:20BA20000198C0B22468A04705E01E48001D077047700021817017480078410008180001A7
:20BA400013490C1802980078207002984078607002988078A07001216078FEF747FB221D90
:20BA600018A003C803C20198A082A5840A2200BF16A116342000FCF78BF806480078411CF5
:20BA8000044A117003B0F0BD0248002141707047340C00205D1B002089BA000831B7000871
:20BAA00081B700086C0F002037B8000843444300434443204441544120696E7465726661DD
:20BAC0006365000000C2010000000800A12000000000020000000000F8B4059C2E4D2E78A2
:20BAE000761C2E70F6B2042E08D2B700BE19AD196D1E2871E9702A70AC706B70F1BC70479C
:20BB000038B50C000021244D2D1D2A79824227D108212000FFF702F80B212000FEF7FEFF7A
:20BB200029792000FEF7FAFFE9782000FEF7F6FF29782000FEF7F2FF69782000FEF7EEFF60
:20BB4000A9782000FEF7EAFF287941000818C000124908182B3001782000FEF7DFFF31BDD4
:20BB6000491C6D1D0329D0DB31BD000010B50A4CFF220F21201DFBF73BFF0020207007483D
:20BB8000C42100BF06A24250001DEF210170022141700121817010BDF00D00206C0F0020BD
:20BBA000D9BA000801BB00087047FEE770B504000E0072B6084D6878401C68700822002177
:20BBC0002000FAF773FC66716878401E68706878002800D162B670BD78010020FEB5060088
:20BBE0000D000A9F44220021FAF760FC341D01982061207B1349097801432173392037541C
:20BC0000002D00D02562089FA762099D65622A00CD213800FAF74AFC7819072188435038F0
:20BC200000210160802149044164074901640299C1640221C943416220603000FAF7DAFD30
:20BC400003B0F0BD5B1B0020EB7A000830B4434351435D18010C0C00130C5C432D1980B2BF
:20BC6000434392B251430024C918644124040B04090C09195043C018694130BC7047124242
:20BC800024D0994228D970B500251B4202D00C00002109E00024012649186441944200D34B
:20BCA000A41A7641F8D33100012601E0764109D2001864416D41A41A9D41F7D2A4185D414F
:20BCC000B619F5D3300022002B0070BD1B42D8D108B500F08BF908BD01D19042D3D20200DC
:20BCE0000B0000210020704710B5040002E0C068FAF742FD72B620680028F8D1024840789B
:20BD0000002800D162B610BD7801002000B585B002900190094A9368039372B60368009395
:20BD20006B4603600098002800D0436090686A4682600174FAF78AFD05B000BD780100203A
:20BD400038B504000B4D2878401C287072B66878401C68702000FCF727F9200000F048F946
:20BD60006878401E68706878002800D162B6FAF7EAFC31BD7801002038B5040072B60E4DEA
:20BD80006878401C68702079002807D148212000FFF7BCFF6079022805D102E060790128FF
:20BDA00001D0002020716878401E68706878002800D162B631BD00BF7801002038B57A4C01
:20BDC000E5690F202062A80604D5A08CC0B2774949688847680613D568467449896888477E
:20BDE00000280AD020684021884320609020C00501686F4A0A40026031BD68460078208511
:20BE000031BD9021C9050A68694B1340802212031A430A60644908850868402202430A6003
:20BE20007047F2B5050017001E00604C2078002801D000F075F8E66067600098A0605D4886
:20BE40000168802292020A4302609021C905CA68594B13408422D2021A43CA608A68574B57
:20BE600013438B604A6A564B13404B624A6A88235B0013434B620A68524B13400B60802200
:20BE8000D2038A610A68504B1340820C1A430A600A68474B13400B600A684C4B134080226D
:20BEA00092031A430A600126C1693143C1614168B2030A4342603C4F002038607860B860BF
:20BEC000F00338604248854200D3451EE80F40194010404940182900FEF7F6FB082801D2BD
:20BEE000082003E03104884200D3481E3A4A02400007400F1043B88138680D2101433960AC
:20BF0000364801680902090AB2070A4302603448F106016038682021014339602670F1BDDE
:20BF200024480168802292020A4302609020C0050168244A0A4002600168234A0A400260CD
:20BF400001681B4A0A4002600168204A0A40026000201549086015490870704780B501221D
:20BF600088216846FDF768F968460078FF2803D068460078012800D0002002BD1A4900286C
:20BF800001D0402001E08020C003086070479020C00501680C4A0A40026070471148008895
:20BFA0000006C00F7047000000380140100B0020FFFFF3FF14100240FF0FC3FF00F03C00EF
:20BFC0000FF0FFFFFF3FFFFFFFCFFFFFFFFFCFFF41420F0000D8B805F0FF000018E400E09E
:20BFE00000E100E010000048180000487047FEE772B60021017103484078002800D162B65D
:20C00000704700BF7801002008B4024B9C4608BC6047C046F105002010B5FDF706F90400E3
:20C020007020FAF749FE70212000FAF7D9FD10BD7047F0B585B007006846002101700020FB
:20C04000C043FBF7D7FB03ACCD2F06D1022103A8FAF750FE2078617805E0032103A8FAF774
:20C0600049FE6078A1780902401880B2C01D0490C6107400601CFBF7EFFD02908019019022
:20C08000029800280CD12000FAF73EFE3000FAF702FE6846062101700121FAF7A1FD50E06C
:20C0A00031000198FAF726FE31000298FAF73EFE0024FAF75BFE311A0D1B002803D0FF2DA1
:20C0C000F7DD3F208543EB00B14204D104984007400FC01F1B1868460078002811D1B54841
:20C0E0000078012814D1B4480021C943016001980219011902980019FCF7B7FF69460870DF
:20C1000006E0DB1DDA10002101980019FAF7CEF9D52F13D02900CF2F0CD1A8484078002811
:20C1200008D06019B04205D1019800196A4612784255491C01980019FAF7B2FD6419B44239
:20C14000B7D19E4C2078002802D1684600782070D52F0AD0FAF7BCFDCF2F06D160780028C7
:20C1600003D168460078FAF7A1FD0298FBF79AFD05B0F0BDF0B583B0032101A8FAF7BAFD64
:20C1800001A805784178807800020C1801202907090F884040100090661C3000FBF75CFD94
:20C1A000070009D12000FAF7AFFD2000FAF773FD0620FAF77BFD3BE0281126D1210038002D
:20C1C000FAF7B4FD0026FAF7D1FD211A8D1B002803D0FF2DF7DD3F2085430098002803D040
:20C1E0006843800AFAF755FB29007019A04203D1B81900224255491CB819FAF751FD7619D3
:20C20000A642E0D1FAF764FD0FE021003800FAF771FD0098002802D06043FFF7F5FE00204E
:20C22000385531003800FAF7DBFC3800FBF73AFD03B0F0BD1CB56C46FCF797FE208000F0E4
:20C24000C1FFA07000F0C2FFE07000F0C3FF207100F0C5FF607100F0C6FFA07100F0C7FFC9
:20C26000E07108216846FAF7BBFC13BD80B50420FAF722FDAD48FAF71FFD80200001FAF721
:20C280001BFD01BD80B5042101A0FAF7A9FC01BD335AEAB800B589B0202200216846FAF75A
:20C2A00005F9A3496846FAF7CFF868461C2101717C214171A12181710221C1712021FAF747
:20C2C0008FFC09B000BD00B583B06846FCF7D9FE06216846FAF784FC03B000BD80B5FCF71F
:20C2E000DEFEFAF7EFFC01BDF0B5A3B0002700260025042101A8FAF7FDFC12E04000401024
:20C300000090FA2189000098201AFAF700F904002000A90002AA50506D1C761C0198400818
:20C320000190019800281BD0C007F6D50D2E03D10220FCF7FDFEECE73000FCF7F9FE04001E
:20C34000B01E022802D919380128E1D8042280216846FCF771FF00980028CFD50097D0E74D
:20C36000A90002A8FAF73CFC23B0F0BD70B5A2B00024002504216846FAF7BCFCA748002175
:20C38000C94301AE0DE0D20706D50A00042C00DA0268AB00F2506D1C641C009A5208009247
:20C3A000001D009A002AEED1A90001A8FAF718FC22B070BD611B0020B8110020561B002071
:20C3C000F0B5C5B002A8FAF7B7FC6846FAF7B4FC01200321029A0A4000D00020009A1140A0
:20C3E00000D000208E490F68002F2BD00021C9438F4227D0002825D002980190009C80205C
:20C400004000844200D904000098001B0090039404AE0198FAF72DF805006F4039003000E1
:20C42000FAF712F87F4F6F40361D0198001D0190241FEED1039904A8FAF7D2FB0098002822
:20C44000DCD102E01046FAF726FC45B0F0BD80B5FBF7F3FBFAF736FC01BD10B5C0B0802473
:20C460006400220000216846FCF77CFF74E0F0B585B00024E44380277F003800FBF7ECFB49
:20C48000050004D186204000FAF73EFC49E03900FAF730FC042102A8FAF72CFC082103A876
:20C4A000FAF728FC00223900280000F0A5FE0299884236D1082203A95B48F9F7E5FF002870
:20C4C0002FD100242E000122210001A8FCF74AFF3078694609790140814220D1641C761C01
:20C4E000BC42F0D328002030F9F7C3FF002816D02800F9F7BEFF040011D004220021684694
:20C50000FCF730FF00980021C943884201D0844205D139002800FCF73CFF040001D5002470
:20C52000E4432000FAF7CEFB05B0F0BDE32E0000335AEAB880B580204000FAF7E5FB002052
:20C54000FAF7B4FB01BD10B5C0B080246400220000216846FCF770FE21006846FAF740FBF3
:20C5600040B010BD10B5040004222021FCF764FE0422242120000830FCF75EFE04224021E0
:20C5800020000C30FCF758FE0422482110342000FCF752FE10BDF0B589B00025ED4380261A
:20C5A00036013000FBF758FB040003D1BF48FAF7ABFB2DE032000021FCF73EFEF708390092
:20C5C0002000FAF797FB04216846FAF793FB082101A8FAF78FFB00223900200000F00CFEA4
:20C5E0000099884211D1082201A90F48F9F74CFF00280AD103A8FFF7B5FF31002000FCF7F4
:20C600009AFE050001D50025ED432000FBF74AFB2800FAF757FB09B0F0BD0000CC0A002034
:20C62000E00A0020A5A5A5A5B0C8000880B580204000FAF769FB01BDF0B5CBB0002701214B
:20C6400002A8FAF757FB6846FAF776FB6846007A002812D06846007A022841D180277F0021
:20C66000082103A8FAF746FB082203A990A0F9F70BFF002804D0002013E180273F01EFE7E7
:20C680003800FBF7E9FA0190002801D03E0003E0802676000AA801903800FAF713FB002428
:20C6A0003500BE4200D93D006846007A002805D12A0021000198FCF7BFFD04E02A00210047
:20C6C0000198FCF74FFE29000198FAF789FA64197F1BE5D101980AA9884200D1E4E0CDE026
:20C6E0006846007A012869D1009880210901884200D0C6E06D48FBF7AFFA040027D0009948
:20C700000C31FAF7F7FA00220099200000F074FD050000982018F9F7ACFE854209D1082284
:20C7200000982118091D00BF61A0F9F7ADFE002802D00020C04306E005A8FFF713FF009956
:20C740002000FCF7F8FDFAF7BDFA200096E005A8FFF708FFFCF796FD00240025009E8020DC
:20C760004000864200D9060031000AA8FAF7C2FA2A0031000AA800F03FFD050032002100B1
:20C780000AA8FCF785FDA4190098801B0090E5D10C210AA8FAF7AEFA0AA8F9F76AFEA842D0
:20C7A00007D108220AA9091D41A0F9F76DFE002802D0FCF767FDFF43380073E06846007A1C
:20C7C0000328009863D180214900884259D186204000FBF741FA060053D000990C31FAF781
:20C7E00089FA00220099300000F006FD050000983018F9F73EFE854209D10822009831181B
:20C80000091D00BF2AA0F9F73FFE002802D00020C04330E0009F002435000122210002A829
:20C82000401CFCF79FFD28786946497A014081421FD1641C6D1CBC42EFD330002030F9F7CE
:20C8400018FE002815D03000F9F713FE040010D00422002101A8FCF785FD01980021C94375
:20C86000884201D0844204D139003000FCF791FD01E00020C043FAF725FA3000FBF712FA56
:20C8800012E000980C30FAF73FFA002009E0002801D00C3000E0082000900098FAF734FA1B
:20C8A0000120C043FAF70EFA4BB0F0BD0C080000494453454747455200B583B0012101A8A2
:20C8C000FAF718FA0090002811D168460079FE2803D0FF2804D1022004E08E48007801E06A
:20C8E00000F0BAFC009004216846FAF779F903B000BD80B502216846FAF7FCF9684600883A
:20C900008549884202D168460021018068460188FA208000484300F014FC01BD80B500F01D
:20C92000B9FC01BD80B500F0B9FC01BD70B584B0012102A8FAF7DEF904216846FAF7DAF968
:20C94000042101A8FAF7D6F900283BD400980199014337D0019EFBF770F9B04202D2FBF7E3
:20C960006CF906003000FBF777F9040002D100F02BFA27E03200AA21F9F798FD019D29007E
:20C98000B54200D931006D1A6846007A642802D0652806D00BE02000FAF7ACF9002808D580
:20C9A0000DE0009820602000FAF71AF901E000F00BFA002DE3D10098401E0090DED1200042
:20C9C000FBF770F904B070BD10B582B00124012100A8401CFAF78EF901216846FAF78AF91D
:20C9E0000220FAF791F9002813D1684640780002694609780843FF21891C884205D093496B
:20CA0000884202D09249884200D1924C2000FAF759F913BD80B504216846FAF76BF96846E8
:20CA200081780902C2781143FF22921C914205D0864A914202D0864A914202D10078F8F79B
:20CA4000A7FF01BD002084490A3104220B88002B00D0401C1C31521EF8D1704701000020DC
:20CA60007D4A0A3213888B4205D0401C1C320428F8DB0020C0437047FFB583B00224764D23
:20CA80000027002628000A30018800291ED1F000801B80002C1804982060059860606846D0
:20CAA000007E20720CA800786072684680896081AD48006AE0606846FAF786F800982061FB
:20CAC000019860613000FAF795FE20E0761C1C30042ED9DBA448006A002629000C31B84B9F
:20CAE0008A1E1288002A0CD00A68821A9A4208DB3000FBF7FFFCF000801B800028184781F1
:20CB000003E0761C1C31042EEADB641EB9D107B0F0BD0000611B0020FFFF000070B59AB0E3
:20CB2000012102A8FAF7E6F8042105A8FAF7E2F8042104A8FAF7DEF8012101A8C01CFAF78D
:20CB4000D9F8012101A8801CFAF7D4F8022101A8FAF7D0F86846007A642802D0652829D04F
:20CB600046E068468088002815D196480188491C0180684681808088FFF770FF0028F4D571
:20CB80006846807900906846C379049A05998088FFF772FF2CE068468088FFF75FFF00288B
:20CBA00026D4C100081A80002B4908186E49096AC1601DE068468088FFF750FF040017D452
:20CBC000E000001B800024490D1800266E81A869002802D0FBF766F8AE612000FBF78AFC31
:20CBE000FFF730FF002803D1FCF7DBF99548066006A803906846818803A8F9F713FC042143
:20CC000003A8F9F70FFC102103A8F9F70BFC042103A8F9F707FC00240F4D10222900039862
:20CC2000FAF7B6FF039810300390641C1C35042CF3DBFCF79AF9010003A8F9F7FAFB2101D8
:20CC40000C3106A8F9F7CCFF1AB070BD0103000001060000FF0500004C12002030B583B092
:20CC6000022100A8801CFAF745F8002401AD19E002216846FAF73EF8022101A8FAF73AF86D
:20CC80000221A81CFAF736F80221281DFAF732F80221A81DFAF72EF801A96846008800F03C
:20CCA00064FB641C684640888442E1DB03B030BD70B583480068002804D12B48006A814901
:20CCC000884201DAFCF7EAF97F4E34687F4D012C24DB08D12869401C2861642803DA0020A0
:20CCE00000F01FFB08E0002000F00AFB002028619A48844200D10124641C3460984884422C
:20CD000019DB64212000F9F7F7FB002803D0002000F0F6FA0FE000F004FB0CE0002C0AD5C8
:20CD2000002000F0FEFA3068401E30608D49884201D1FCF7EBF9FCF718F98B4988422868EA
:20CD40000AD38A4988420CDA002802D16868401C686028680A3005E0002802D06868401CAF
:20CD600068600020286070BD7801002038B5804C2068401C20600A2811D17E480168491CB8
:20CD800001607D484168491C416000252560FFF78FFF6068401C60600A2800D1656000F0F4
:20CDA00095FAFCF7E2F875490A68904200D802000A604A68824200D202004A6031BD0000EF
:20CDC00010270000541B002072B6002000F0BAFAFAE780B5FFF7F8FF01BD80B500F052FA6F
:20CDE0000220F9F756FD00F051FA01BD80B500F051FA0220F9F74DFD00F050FA01BD70475A
:20CE000080B500F0AFF900F0E5F9F9F74FFF01BD80B5CD20FFF70DF901BD80B5CE20FFF786
:20CE200008F901BD80B5CF20FFF703F901BD80B55348012141705348F9F77EFF5248F9F72A
:20CE400041FF01BDCC12002010B584B00124E44310216846F9F74EFF0098802804D20199C5
:20CE6000FCF7BAF9040026E0C021490088420BD28039884202D1019844491AE0491C88428C
:20CE800019D10198424914E08031884213D27F39884207D168460089FFF7E0FD0199FAF741
:20CEA000C0FC00240098C1214900884203D101983849086000242000F9F704FF04B010BDF7
:20CEC000BC120020C0D4010048120020CC0A002070B50400304D2868002813D1601F0FD0BF
:20CEE000C2380DD0801F022805D90838012802D9C01E05D006E029492948007800F01CF977
:20CF0000012028601B2C04D3BA2C01D2FFF75CFF61342406A00D00BF26A1085880472148BE
:20CF2000006A00240025204E31000C311F4A8B1E1B88002B0CD00B68C31A934208DB280076
:20CF4000FBF7D8FAE800401B80003018448170BD6D1C1C31042DEADB70BD0000FFFFFF7F9B
:20CF6000B30200000CFEFFFF4C040000005C2605E40A0020C012002000010020C412002006
:20CF8000561B00203C120020104704004012002044120020E00A0020CC12002040420F00B6
:20CFA000611B0020780100204C120020C027090070470000D3CD000819C00008DBCD0008DE
:20CFC000EDCD00086DC20008F3C800080192000835C20008D3CD00081DCB00085DCC000832
:20CFE000FFCD000821E200082FCE000849CE0008D3CD0008D3CD0008D3CD000897C50008D2
:20D000006FC40008D3CD0008D3CD000839C60008D3CD0008D3CD0008D3CD0008D3CD0008DE
:20D02000D3CD0008D3CD0008D3CD0008D3CD0008D3CD0008D3CD0008C7C20008E9C20008BC
:20D040006DC300082DC9000833760008F5760008B9750008B9C8000801CE00087DD100088A
:20D06000ADD1000875D10008A5D1000811CE00081BCE000825CE0008D3CD0008D3CD00083B
:20D08000D3CD0008D3CD00084FC40008D3CD0008D3CD0008D3CD0008D3CD0008D3CD0008DD
:20D0A0006DD100089DD100081DC9000825C9000885D200088DD20008D3CD000873A2000845
:20D0C000D3CD0008D3CD0008D3CD0008F77500085BC4000835C5000885C20008C9C90008D2
:20D0E00015CA000883D50008D3CD000895C20008D3CD000875C10008DDC20008D3CD0008AD
:20D1000047C500082DC60008D3CD0008D3CD0008D3CD0008D3CD0008D3CD0008D3CD000810
:20D12000D3CD0008D3CD0008D3CD0008D3CD0008C1C30008D3CD000880B5FBF7B9FF00201C
:20D1400002BD80B5FBF77AFF002002BD80B5FBF772FF02BD80B5FBF72FFF01BD80B5FBF700
:20D160003DFF01BD80B5FBF760FF01BD80B5FBF74CFF01BD80B5FBF746FF01BD80B5FBF7F0
:20D1800031FF01BD80B5FBF72CFF01BD80B5FBF71CFF01BD80B5FBF722FF01BD80B5FBF764
:20D1A00039FF01BD80B5FBF72FFF01BD80B5FBF71EFF01BD80B5FBF713FF01BD80B5FBF746
:20D1C000EEFE02BD80B5FBF7D7FE02BD80B5FBF7D8FE02BD80B5FBF7D6FEC0B202BD80B5CC
:20D1E000FBF7C5FE02BD80B5FBF7D2FE02BD80B5FBF7D3FE02BDFEE7F0B491B00300100071
:20D200000F226C463C3416000425F707FF0F7608002F02D037000F4E7E406D1EF5D12660C8
:20D22000521E241F002AEED51A7842405B1C1007800E6C462458100960400207920E6C46DC
:20D24000A25800095040491EEED111B0F0BC7047000000002083B8ED70B50400074D28788C
:20D260000600012803D1012C01D000F025FA04492000FFF761FF2C70300070BD611B002046
:20D2800040420F0080B5FFF769FF01BD80B5FFF781FF01BD80B5FFF75DFF01BD80B5FFF7D3
:20D2A00075FF01BD80B5810009184900414A51180A78002A01D0897800E04978002902D00E
:20D2C000FBF74BFF01BDFBF751FF01BD70B50024384DAE88002E0FD0761E012E0BDAA8787B
:20D2E000002801D02E8900E0EE8801214140A9702000FFF7D7FFAE800A3D641EE9D570BD9E
:20D30000012800DB704780B5810009184900294A511801224A700978002901D1FBF71DFFEF
:20D3200001BD012800DB704780B5810009184900204A511800224A700978002901D1FBF737
:20D3400015FF01BD012800DB704780B5810009184900184A51184A78012353404B700978A0
:20D36000002901D1FFF79EFF01BD012800DB704710B58200121852000E4B9A180B881370C2
:20D380008B88D380CB881381CB88002B08D08C88002C01D1002304E04C88002C01D02300DD
:20D3A0000124938094700988002900D19180FFF779FF10BD200B00207047FEE7F1B584B099
:20D3C0000026BC4C2068002806D101960296082101A8F9F705FC5AE003A9684600F0F9F930
:20D3E0000098A168451A05D10398002805D1E568012602E001D5E0682D180498854200DAC8
:20D400000495019604980290082101A8F9F7E8FB0498002839D0A068009A90421FD362680C
:20D42000151A04998D4200DD0D002E0013D03100F9F736FCF9F7A0FC371AFBD0A068C0197A
:20D44000A0606168884201D32068A060A06800F0C8F9F61BEED10498401B049015D0049D43
:20D460002900A068F9F71CFCF9F786FC2E1AFBD0A0688019A0606168884201D32068A0605E
:20D48000A06800F0AEF9AD1BEED1F9F721FC05B0F0BD38B5874C05E06846017820001430C7
:20D4A000FAF740FD01216846FAF73CFD6846007800282FD1606900F0B9F905006968286825
:20D4C000F9F720F8A169884200D90800A061A9682868F9F717F8A169814200D20100A1614C
:20D4E0002068002807D0E168226991423BD0FAF7D9FB002020602069002829D1754DFAF730
:20D500009CFB401905408020800085421FDA0020C04333E0012100A8401CFAF703FD6846FB
:20D5200040780128B8D0022802D0042805D009E06846017820001830B2E76846017820002D
:20D540001030ADE768460078F9F7DEFBAAE725612069FAF781FB20602069E0602168081809
:20D560006060002909D000F024F923692268A169606900F0CEF82068A0600020F9F7A2FB08
:20D5800031BD10B588B0012100A8801CFAF7CAFC68468078662820D10020019002E001A822
:20D5A000FAF7C0FC01216846FAF7BCFC68460078002804D10198FFF701FF08B010BD0121EC
:20D5C00000A8401CFAF7AEFC6846017840780328E5D00800F9F798FBE4E768468078642865
:20D5E00004D065280ED06E2823D0E6E7FFF751FFE3E7012100A8401CFAF794FC68460078B9
:20D60000F9F782FB01216846FAF78CFC684600780028EED1274C2068002806D000F0C9F89D
:20D620002068FAF73FFB002020600020F9F74AFBC3E70020019002E001A8FAF773FC0121DA
:20D640006846FAF76FFC68460078002824D10198002802D00020C043E8E700F0E7F8010028
:20D66000142202A8FAF7A8FA1C20F9F7D7FA0198F9F7D4FA0298F9F7D1FA0398F9F7CEFA3B
:20D680000498F9F7CBFA0598F9F7C8FA0698F9F7C5FAF9F71DFB90E7012100A8401CFAF707
:20D6A00041FC6846017840780128C5D00800F9F72BFBC4E77402002010B5074C2068002869
:20D6C00006D000F076F82068FAF7ECFA0020206010BD000000FEFFFF74020020474801899F
:20D6E0000F220368134001D04260704744484269002A0DD0026911700169491C0268436803
:20D70000D318994200D1110001614169491E4161704770B53A4881610260436039498024E1
:20D7200064024A6922434A610A68630013430B60354D00262E6001680161416841618660F8
:20D74000C66081694808314A8018FCF7D1FF082801D2082002E0A04200D3601E9021C905D4
:20D760008A68C02313438B600A68C0239A430A600A68802313430B600A6A254B13400B627D
:20D780000A6A230913430B626E60AE60214A02400007400F1043A8811F4828601F4801680C
:20D7A000FF22914340220A4302601D482103016070BD154801682422914301601948016841
:20D7C000802292020A4302600168174A0A400260704772B60A4A53690B601169016062B6A1
:20D7E000704772B606490A69824201D2801A02E04B689A1A1018486162B670471C440040CE
:20D80000F40A00201C1002400044004000D8B805FF0FFFFFF0FF0000258000001CE400E0E3
:20D8200000E100E010100240FFFFFDFF00A07047006CDC02C0000000FFFF0000000000006C
:20D8400000000000016800E0491C0A78202AFBD0092AF9D00D2AF7D00A2AF5D00160704778
:20D86000F8B504000F0000260025FFF7EBFF206801786A46437813701A020A43A04B9A429E
:20D8800034D1801C01780A00303AD2B20A2A01D230390CE00A00413AD2B2062A01D237399E
:20D8A00005E00A00613AD2B2062A3ED2573900293BD4401C2A01551801780A00303AD2B2ED
:20D8C0000A2A01D230390EE00A00413AD2B2062A01D2373907E00A00613AD2B2062A01D35A
:20D8E00020601AE057390029E3D5F9E72D2917D10126401C69460978401CAA0052195200A9
:20D900003039551801780A00303AD2B20A2AF3D32060002E01D0280045423D600020F2BD2C
:20D920000A00303AD2B20A2AE6D30020C043F2BD7047B448006A704780B501000868496805
:20D9400000916B4600220421FAF763FE002802D50020C04302BD002002BD80B50100086886
:20D96000496800916B4600220221FAF752FE002802D50020C04302BD002002BD80B5010038
:20D980000868496800916B4600220121FAF741FE002802D50020C04302BD002002BD80B5BB
:20D9A0006B46002204210068FAF708FE002802D50020C04302BD009802BD80B5FAF75CFE58
:20D9C00002BD80B5FAF771FE02BD80B56B46002202210068FAF7F2FD002802D50020C0439F
:20D9E00002BD009802BD80B56B46002201210068FAF7E4FD002802D50020C04302BD009834
:20DA000002BD80B54168006808280CD0092811D00A2817D00B281DD00C2823D00D2829D055
:20DA20001C282FD033E0FA20800041430800FFF788FB2CE0002902D0FFF7A8FB27E0FFF754
:20DA400089FB24E0002902D0FFF7B4FB1FE0FFF799FB1CE0002902D0FFF7A0FB17E0FFF7A0
:20DA600085FB14E0002902D0FFF7A0FB0FE0FFF785FB0CE0002902D0FFF794FB07E0FFF7F8
:20DA800079FB04E0481E8041C00F94490870002002BD80B5006808280CD0092811D00A2817
:20DAA00012D00B2813D00C2814D00D2815D0162816D018E0FFF74AFBFA218900FCF718FE38
:20DAC00002BDFFF790FB02BDFFF791FB02BDFFF779FB02BDFFF783FB02BDFFF777FB02BD83
:20DAE000C148007802BD002002BD01218143BF480170704701218143BD48017070470000DF
:20DB000030780000F0B583B000680190081800906846FFF797FE02E00098401C00900098A5
:20DB2000017800295FD0401C0A00613AD2B21A2A06D30A00413AD2B21A2A01D35F294FD1A9
:20DB4000012601E0761C401C01780A00303AD2B20A2AF7D30A00613AD2B21A2AF2D30A0024
:20DB6000413AD2B21A2AEDD35F29EBD0002E37D025A5002707246868B04208D132000099A8
:20DB80002868F8F781FC002801D1012702E00C35641EF0D10098801900906846FFF752FE4C
:20DBA000009800783D281BD10098401C009001A96846FFF755FE002F04D0A968080001D0F2
:20DBC000019888476846FFF73DFE00980078002809D06846FFF736FE009800783B289BD037
:20DBE0000020C0430BE0814C2078002805D17E480078012801D1F8F7AFFA0020207003B080
:20DC0000F0BD000078010020DCF300080500000031D90008E4F300080500000031D90008DA
:20DC2000ECF300080600000031D90008F4F300080600000031D90008FCF300080B000000DC
:20DC400031D9000808F400080E000000EBDA000818F4000813000000F5DA000800207047FE
:20DC6000A348704780B50068F8F713FE02BD80B5FFF770FA02BD80B5FFF788FA02BD80B5B1
:20DC80000068FFF7E9FA02BD10B50C00C368816862184168611800682018FBF7E6F910BDC5
:20DCA00080B50A00416800681018F9F723F802BD80B50A00416800681018F8F791FF02BD6C
:20DCC00080B50068FFF73DFA02BD80B50068FBF7F1F802BDB448006A70470000621B0020CA
:20DCE00080B50068002802D0FFF758FA02BDFFF73DFA02BD80B50068002802D0FFF756FABD
:20DD000002BDFFF73BFA02BD80B50068002802D0FFF748FA02BDFFF72DFA02BD78B402685A
:20DD20008A1843688168C068DC0812195B075B0FFF25FF249C40C018083803D54642354199
:20DD400025402C001578A5430E009E4034402C431470012801DA002013E0521CD94008289C
:20DD600007DB08381170521C090A0828F9DA002807D001248440641E1078A0430C40044314
:20DD8000147072BC704710B582688C18416802680120C043144B1B78002B0FD0012B0DD18A
:20DDA000002907D0002104201043F8F77FF92100032001E021001000F8F778F910BD10B51C
:20DDC0008168436802680120C043074C2478002C09D0012C07D1002B02D00420104300E0D4
:20DDE0001000F8F710F910BD611B00205C1B0020601B002080B502689D48007800280CD080
:20DE000001280AD1002104201043F8F74FF969460320F8F74BF9002802D50020C043009078
:20DE2000009802BD80B5006891490978002906D0012904D16946F8F739F9002802D50020A6
:20DE4000C0430090009802BD416802680120C043874B1B78002B00D1704780B5012B03D154
:20DE600004201043F8F7CFF802BD416802680120C0437F4B1B78002B00D1704780B5012B0E
:20DE800002D11000F8F7BFF802BD80B50068C0B2072805D28000774908588047FF2801D1C5
:20DEA0000020C04302BD1248704711487047104870470F48704780B50068FDF70FFB002087
:20DEC00002BD80B5FDF749FB002002BD80B50A00416800681018FDF793FB02BD80B50A003F
:20DEE000416800681018FDF74CFB02BD00487047FAFEFFFFF7B5060000200090C800401A76
:20DF00008000C44908188769002F01D1042037E03868C149884206D101220092BA68CE2A0E
:20DF200001D301202CE0884221D13C002034F868C000381820300190002501E008346D1C78
:20DF4000F86885421BDA02992068019A1018F8F7F7FA0028F2D1646850213000F9F766FD34
:20DF600045A0F064009800280CD038690AE0AB490298F8F7E5FA002801D10424ECE70320CD
:20DF8000C0430FE03818B0643464B06C0268F2630099002905D0121FF26304218018F8F7EF
:20DFA00053FA002003B0F0BD78010020F5B581B0C800401A8000974908188669002E01D18F
:20DFC000042039E00020009030689349884206D101220092B268CE2A01D301202CE08842AD
:20DFE00021D134002034F068C00037182037002501E008346D1CF06885421CDA02992068E6
:20E000003818F8F79DFA0028F3D1646850210198F9F70CFD019800BF17A1C164009800287A
:20E020000CD030690AE07D490298F8F789FA002801D10424EAE70320C04316E030180199BE
:20E040008864019804640198806C02680199CA630099002906D0121F0199CA6304218018D0
:20E06000F8F7F2F9019800F0ABFA03B0F0BD0000611B0020B801002077DC00086FDC000815
:20E080007FDC000889DC0008C1DC0008CBDC000861DC0008A1DC0008B1DC0008D5DC000844
:20E0A000E1DC0008F5DC000809DD00081DDD0008BFDD000887DD00088BDE000861DC00080C
:20E0C00061DC000861DC000861DC000861DC000861DC000861DC00087DD900085BD9000808
:20E0E00039D90008E7D90008CBD900089FD90008BBD90008C3D9000803DA000893DA000878
:20E100005DDC00085DDC000861DC000861DC000861DC000861DC000861DC00085DDC0008E3
:20E120005DDC000805DB000865DC00085DDC00085DDC00085DDC00085DDC000861DC000824
:20E1400061DC0008A7DE0008ABDE0008AFDE0008B3DE0008B7DE0008C3DE0008CDDE000835
:20E16000DDDE0008EDDE000849DE0008F5DD00086BDE000825DE00085DDC00085DDC000822
:20E18000F0B585B00F0015000B2804D110216846F8F7B0FD06E00C216846001DF8F7AAFD8A
:20E1A000002000900098C0B2009002981A49884200D1039801994418164E0098C100081A0D
:20E1C000800030188069002808D0F9F76BFD0098C100081A8000301800218161603420003C
:20E1E000F9F73AFD04000CD0082269460831F9F7CFFC0199083920000830F8F77BFD3C6015
:20E2000003E001980838F8F77FFD0098286005B0F0BD00004C12002050435632A8E3000829
:20E2200030B5A3B0012104A8F8F764FD6846007C0A2800D9AEE002A1095C49008F4400BFE2
:20E2400006080DAAAA3E6472AA899A00534801E000F0D0F9F8F736FD9CE06A4601A902201F
:20E26000FFF78EFF4E4C0098C100081A8000201801998161484D00BF4BA200992800FFF7DA
:20E2800095FE0990286C0A9028680B90E86B0C90686C0D900098C100081A8000201880697D
:20E2A000002808D0F9F7FEFC0098C100081A8000201800218161142109A869E000250024C6
:20E2C0006A4601A90520FFF75BFF0420019900290AD00099CA00511A8900314A5118019AD8
:20E2E0008A610290039502E00290E4430394082102A8F8F775FC002C4CD400BF2AA20021AC
:20E300002548FFF7F7FD45E0254CA0690025002802D0F9F7C7FCA5610420029003950821B8
:20E3200002A835E0082105A8F8F7E4FC1A4D1D4B069A0599280000F0A9FA4C210E910F9006
:20E34000482229000EA80830F9F736FC50210EA81EE00C2105A8F8F7CDFC042105A8001D74
:20E36000F8F73EFC069905980B4A926C1018F8F737FC0FE00C2105A8F8F7BCFC06990598EF
:20E38000054A926C1018F8F7B5FC042105A8001DF8F726FC23B030BD780B0020E607000018
:20E3A0004C12002033D900086D61696E00000000012000BD022000BD0A0B9200A3585B1E4E
:20E3C000A35002D00A05120EB61AB95BB61CCA06520EA85887460A0552160B0B9B001959FC
:20E3E00089181951F1E70A05120F92000B0B9B00E3580906090F5918A150B95BB61CCA064D
:20E40000520EA858874660B40E0BB600A65901E060B40E0B0B051B0F9B00E5580906490F66
:20E420008900734808588746AD19E550002D03D10122626460BCC8E70022626460BCC4E70C
:20E44000AD1BF2E73540F0E73543EEE77540ECE7B540EAE7F540E8E77543E6E70A0B920004
:20E460000905490EA150B0E70A0B9200B95BB61CBB5BB61C1B040B43A350A6E7626CD207A6
:20E4800003D5A2E7626CD2079FD509040916490076189AE7626CD207D20F090B89006250A5
:20E4A00093E7CA09E36BF8184906490F8900C918E1633900E36C9A5800F002F8206084E70D
:20E4C00010478A0603D5E26B121FE263BE50090489154900761878E78A0603D5E26B121FE5
:20E4E000E263BE50090B890066586EE70A05130F9B00E3180A0B9200E06B801A19003B185A
:20E50000E06308681860091D1B1D121FF9D15CE70A05130F9B00E3180A0B9200E06B39182A
:20E520008018EDE7E26BD659121D490989005218E2634AE7CA12D2065216E36BD2188B0525
:20E540001B0F9B00490502D5E358D3513DE7D259E2503AE720B44806420F0D052D0FAD0062
:20E56000080B800020180368FB1809061CD5110003D11878605120BC27E7012A03D11888A3
:20E58000605120BC21E7022A03D11868605120BC1BE701784907490F0068C0083818F7F748
:20E5A0002DFF605120BC10E76059110002D1187020BC0AE7012A01D11880F9E71860F7E7EE
:20E5C000F0B5A0B0040000AD266C07498022043A8B58AB50FBD100F003F8266420B0F0BD37
:20E5E00000B5A76CF1E60000D4010020CBE3000854020020CD207047016C891E016401201D
:20E600007047016C891E0164022070470A0B9200801802680905491651180160002070473A
:20E620000A0B9200821813685B1E136004D0026C0905090E511A01640020704718B40A0648
:20E64000520F0B051C0F0B0BC90601D499004358A10041180C68002A01D1E31819E0012AA7
:20E6600001D1E31A15E0022A01D1234011E0032A01D123430DE0042A01D1634009E0052A77
:20E6800001D19C4004E0062A01D1DC4000E05C4323000B600021002B00D1012141640020B9
:20E6A00012BC70470A05120F92000B0B9B00C3580906090F59188150002070470A0B920060
:20E6C0000905490E81500020704710B4026C836C9B181C885B881B042343121D0264090BA4
:20E6E00089004350002010BC70474422825CD20705D5026C09040916490051180164002093
:20E7000070474422825CD20705D4026C09040916490051180164002070470913890002001D
:20E7200044321278D307DB0F43500020704710B504000A00E06B5106490F89004118E163B8
:20E74000A16C0818520A9200E36C9A5890472060002010BD18B48A0605D5C26B121FC26360
:20E76000836C046C9C50026C89098905491551180164002012BC704718B48A0605D5C26B8C
:20E78000121FC263836C046C9C500913890041580164002012BC70470A0B9200C36B9B1A06
:20E7A000C3630905090F89004118806CC0180B680360091D001D121FF9D10020704718B4B0
:20E7C0000A0B92000905090F89004118C36B846CE4189B18C36320680860241D091D121F0F
:20E7E000F9D1002012BC704710B4C26B836C9B18C9081C240C40241D1119C1631968016445
:20E80000002010BC704770B504004806420F0805050F080B80002058A36C1E18090614D524
:20E82000002A01D130780DE0012A01D1308809E0022A01D1306805E04107490FC008181896
:20E84000F7F7DCFDA90060500AE0A8002058002A01D1307004E0012A01D1308000E03060F1
:20E86000002070BDCA12D2065216C36BD218836C9A188B051B0F9B00C018490502D50068BC
:20E88000106001E01168016000207047F4B5A2B006000C001F00802212A101A8F9F78CF9D7
:20E8A000B06C00902298002802D0B84722994518306C0099095A801C30643000CA06520EB9
:20E8C00001AB9A58904700280AD1002C01D0641E05D022980028EBD0B847281AE8D10020B5
:20E8E00023B0F0BDF9E500083DE6000803E700082FE7000855E70008A5E60008BDE60008F5
:20E9000099E7000807E800080DE6000821E60008E9E7000865E800081BE7000803E6000846
:20E9200003E60008F9E500083DE60008EBE600082FE7000879E70008A5E60008CBE600082A
:20E94000BFE7000807E8000803E6000803E6000803E6000803E6000803E6000803E600086C
:20E9600003E6000878B4C300534C002A246804D0E318524C1B19198012E0E318504C1B196B
:20E98000002501263F2902D24C080E4002E04C090125E10600D0641CE903A4020C431C803C
:20E9A000400080188000BE490B5071BC70478000A54A1018C0229201036813408B4200D151
:20E9C000704730B482B000910368009C634000939E4B009C1C430094BD4C14E080009A4AC3
:20E9E00010183022036813408B4200D1704730B482B000910368009C63400093934B009C2C
:20EA00001C430094AC4C009D25400095009D056005682A408A420CD000910168009A5140CE
:20EA2000009100990B43009300990C4000940099016033BC704710B584B083480168A54A96
:20EA40000A4002609648006800888205920D080518D5A148006802A9022A06D303880B8005
:20EA6000801C891C921E022AF8D2002A01D00088087002A8FCF73AFBC02189010020FFF761
:20EA800096FF16E0002A14D01000934909686B46022808D30C881C80891C9B1C801E022876
:20EAA000F8D2002801D00888187069460020FBF72FF804B010BD0000505C00400260004084
:20EAC00006600040F8B5604C606C9E21090201404A053AD5AB4860649C20000220640020E9
:20EAE0002065AC4D402129617B4F39006C4A202308601060121D091D5B1EF9D1286929691E
:20EB00000A312961216DA44A89180880A34E088880193860002208210020FFF723FF2869C5
:20EB200029690A312961216D89190880088880197860012208210020FFF714FF98482060F0
:20EB40008020E064FBF756F9F1BDCA0411D595486064A16CC02000020840E10B88420CD0C4
:20EB600000286FD0206C0C2188432064FBF764F9F1BD0A050CD58C486064FBF755F9206CD5
:20EB8000082101432164206C042101432164F1BD0A0451D50607360FC106C80F002E0AD12E
:20EBA000002802D0FFF747FFF1BD2068A0490140216000203DE0B10061180028086834D03B
:20EBC000444A02400A60610C3000FFF7F0FEF1003348405800888205920D412A01D3402227
:20EBE00001E0002A17D010003B4B5958694D2B001433022808D30C881C80891C9B1C801E85
:20EC00000228F8D2002801D008881870143529003000FAF77DFF5F48805D002812D0C02171
:20EC200089013000FFF7C3FEF1BD814A02400A603000FBF763F8F1BD880501D5A74800E0E1
:20EC4000A7486064F1BD0000005C00408080000038B505000C00002D16D0FAF70BFD0006A7
:20EC600008D5002C01D0102100E020212800FFF7B5FE31BD002C02D08021490101E080213E
:20EC800089012800FFF793FE31BD80B595490020FFF7A4FE01BD80210143934801607047EC
:20ECA0001C0D002010B5040080218901FFF77FFE8E480021015510BDBF8FFFFF10B5040075
:20ECC000C0218901FFF773FE88480121015510BD8FBFFFFF8F0F00009C0C0020F8B5844822
:20ECE000B830009040688047824C032020640120206400266664800220647F48009909684C
:20ED000088479C20000220642665224D40202861264F38007949202206600E60091D001D37
:20ED2000521EF9D1286929690A312961216D1A4A89180880194E0888801938600022082123
:20ED40000020FFF70FFE286929690A312961216D8919088008888019786001220821002083
:20ED6000FFF700FE0E4820608020E064FBF742F8009880688047F1BD80B55D48EC30006866
:20ED8000804701BDFFFBFFFF5D490878401C0870C0B270479C0D00200460004000600040C6
:20EDA00030320000FFEFFFFFFFF7FFFF9C0C002070B5427953065B0E0188D20900240079A6
:20EDC000002804D0012805D0032805D006E08024A40003E0802400E0C024E400002A01D0E1
:20EDE000202001E080208001204318439C00414D28513E4D2C692E69881C30182861DD0067
:20EE00004048414E002A366802D075192D1802E075193E4EAD192C805C00A418A4003C4EBA
:20EE20002D88281830511800FFF79CFD70BD00000F8F00007047002801D0402070470820FB
:20EE40007047F5B581B00C00C7003148C01945681646E0070BD5022A12D32000FBF7D3F83D
:20EE60002880AD1CA41CB61E022EF6D208E0022E06D320882880A41CAD1CB61E022EF8D2FD
:20EE8000002E01D0207828801C48C01940680299018030210198FFF7A1FD03B0F0BD80B51F
:20EEA000FAF7ACFE01BD80B52021FFF797FD01BD0020704710B50400FAF7DCFBA1000D4ADB
:20EEC00051180A68000601D5402001E08020C001024201D01043086010BD0000FFFDFFFF42
:20EEE000FF61FFFF101000004C5C00409C0D00206C0F0020005C0040C5EA00081C0D0020AC
:20EF00005F1B002000600040505C0040046000409C0C0020FEE7000030B483B05048016862
:20EF200001220A43026041684E4A0A40426001684D4A0A40026001684C4A0A4002604168D2
:20EF40004B4A0A404260C16A0F229143C162016B484A0A400263416B0122914341630021C8
:20EF6000816001910091110402680A430260A023DB014A00046814400094019C641C019470
:20EF8000009C002C02D1019C9C42F3D103689B03DC0F0094384B1124009D012D1C6023D11C
:20EFA00041684160416841604168344A0A404260416822040A4342600168802252040A433E
:20EFC00002608021890402680A40FCD04168032291434160416802220A4342600C2142684B
:20EFE0000A40082AFBD10CE0436B19434163416B1140FCD0416803229143416041680A432D
:20F00000426003B030BC704730B51D4C20680C210140082902D00C2916D017E0206822688D
:20F020000F21850C0D40AD1CC0204002104003D11448454328000AE0A26A13481140491CA0
:20F04000FBF756FB684302E0104800E00E481049086122681206120F8A5CD040086130BD81
:20F06000001002400CB8FF08FFFFF6FEFFFFFBFFFFFFC0FFACFEFFFF00200240FF7FC0FF85
:20F080000410024000093D0000127A00006CDC0218030020F0B586B00200083201688900BA
:20F0A000511800914068C107C90F0591012188438000009908180490002400210026002330
:20F0C00001200290019003E00027019785421AD10098049DA84202D1284606B0F0BD056864
:20F0E000001D03900598002801D048462D18039800682818039F3F1D0097E7E7116854186C
:20F100005168611808328C42F8D0029F002F0ED0267876B2641C002702970127019704E095
:20F12000116854185168611808328C42F8D0002E14D5019F002F01D02378641C8542C3D0BC
:20F140002B706D1C761C0BD5F8E78542BED08C42BCD02378641C2B706D1C761E002EF4D5C1
:20F1600001270297B2E7FEE782B0FAF707F8264A811A491C1000F8F7B3FDF9F7E1FEFEF74B
:20F180001BF90020FEF7BCF8F9F70BFF1F48FDF7D8FFF9F7EAFE0120FCF74AFFF7F7F2FD54
:20F1A000FDF706FFFBF7E8FA194C1A4F1A4D012606E0FEF7C7F8002028603220F7F769FB40
:20F1C000F7F7FEFD0028F4D0144806600020FEF797F810E026606846F7F7F6FD00280AD4E9
:20F1E0000020C0432060FBF7BCFA68460078FDF76FFEFBF7B1FA38780028EBD0F7F7D3FD4F
:20F2000000202860DCE700BF681D0020204E000048120020641B0020CC120020BC120020AC
:20F2200010B5254C2078401C2070F9F795FFFDF79DFD00F049F872B62078012804D160684B
:20F24000002801D0F8F775FC2078401E207062B610BD38B572B6184C6078401C6070FFF777
:20F26000D3FE16480068FA218900FBF741FA8021490488421DD2124A491E0840401E506066
:20F28000104803680B40C0252D061D430560002393600723136002681140802212060A430E
:20F2A00002606078401E60706078002800D162B631BDFEE730BFFDE7780100202803002073
:20F2C00010E000E020ED00E038B5154B1A1D2833D868002803D001201874507017E0D469B6
:20F2E000641CD46103CB083B0025401C694103C3083B106A201A01D401205070187A0028F0
:20F3000005D0401E1872000601D1012010700548046802E0606880472468002CFAD131BD1C
:20F32000780100204C0B002000B583B072B60F484178491C4170FBF713FBF7F796FAFFF713
:20F3400088FF0B4802210291C021C90001910090084B032209A154020019FCF73FFC064844
:20F3600001210170F8F7C7FB03B000BD780100201015002069F100085A1B00204A2D4C69D8
:20F380006E6B0000DDEC000889ED0008B1ED000835EE000879ED000837EE0008B1EE000832
:20F3A00097EC000851EC00088BEC0008A5EC0008BDEC00089FEE000843EE0008A7EE000849
:20F3C000B5EE00080000000000000000000000000000000000000000000000004952507225
:20F3E0006500000044525072650000004952506F737400004452506F7374000049524C6522
:20F400006E44657669636500506572666F726D544946496E6974000052657472794F6E49C0
:20F420006E76616C444150526573700053454747455200004A2D4C696E6B0000577F00080C
:20F44000617F0008257F0008497F0008697E0008C37E0008E57E00087B7E0008A37E00087B
:20F46000A57F000810B5074979441831064C7C44163404E0081D0A68891888470100A1421A
:20F48000F8D110BD0800000038000000136FFFFF70150000F805002004000000681D0020CB
:20F4A00000000000F1FBFFFF0200000002000000B20000001A04000008010020EE04000073
:20F4C000080C10141820303100040C1014181C24282C3034FFFFFF383900000000F009F8B8
:20F4E000002801D0FFF7BEFF0020FFF71DFF00F002F80120704780B500F002F801BDFEE7AA
:20F500000746384600F002F8FBE7FEE701491820ABBEFBE7260002000148804701480047DA
:20F5200019EF000829F50008C046C046C046C046FFF7D4FFF1A0000000000000FEE7FEE759
:20F54000FEE7FEE7FEE7FEE7FEE7FEE7FEE7FEE7FEE7FEE7FEE7FEE7FEE7FEE7FEE7FEE75B
:20F56000FEE703B80B0000FA3005313233343536FC000F661301012CF4000834F400080C92
:20F580000100208F000040E6007EEFD10008CDD10008DFD10008C5D10008BDD10008D5D117
:20F5A0000008E7D10008B1E3000807E400087DE40008A3E40008C3E40008E7E300085DE43A
:20F5C0000008EDE4000855E50008D7E30008B9E3000825E5000835E5000895E40008B5E355
:20F5E0000008B5E30008B1E3000811E4000885E40008A3E40008D9E40008E7E3000869E4E6
:20F60000000811E5000855E5003C08B5E30008B5E30008B5E30008B5E30008B5E30008B591
:20F62000E30008B5E3000829E4000841E4000845E4000849E400084DE4000851E4000855CC
:20F64000E4000859E40008EF000010FA00068025000081C003FB000981E003000020000009
:20F66000FFE0FCFF110000A58D95BD87AFB79F81A9B199A38B93BBF9FF019EE7F9FF01B672
:20F68000EDF9FF020000A5F800E4FFFC0000F0FD0000FFF90001FFE0FBFF0000F8FFF80059
:20F6A0007E0102030406070809006CDC0208B4024B9C4608BC6047C04623D3000808B40242
:20F6C0004B9C4608BC6047C04601D3000808B4024B9C4608BC6047C04637A90008974898F5
:20F6E0004901607047F8B40023944C994D25600026F6430700001D3F68B74201D000200873
:20F70000E05B1CA70DBB4201D125600023091FF0D10120F2BC7047F7B584B0EFF3108002A4
:20F720007E9072B6002001908B480068C0070BD489480068012101438748016086480068FC
:20F740008007FBD5012001907F4C002B49D004987E4901400202120A914242D17C4F06997D
:20F760004118491EC90A39400091C00A0740B94237D3F802802109054618704DE0680006C4
:20F7800003D575482060754820600020E060A069400705D473482860062068607248A8609B
:20F7A0007EE10C3000FFF79FFF002814D10220E0602661E06840210143E160FFF790FFA0D1
:20F7C00068C107FAD4E16802229143E1601421014001D01420A0607F1CE00C36180098B809
:20F7E00042CCD2069840100599049AE3681B0603D55A4B23605A4B23600023E360A3695B9E
:20F800000706D44E4D574B2B6006236B60564BAB600123E3604B4B494D0E88534FBE4211C3
:20F820007ED01788B74200D01680921C891C2B60A668F707FBD41427374006D0A0681421FE
:20F840000143A16003E0921C891C401EE5D10120C043E1680140E1600199012904D13E490A
:20F86000096808403C490860029880F31088069A05990498FFF72CFF002804D107B0F0BDE1
:20F880000020FFF715FF06984400012CF8DB0020FFF716FF641EFAD1F2E7F0B583B0EFF351
:20F8A0007E1081019172B60021002601272A4C22683A4007D122683A432260022223681373
:20F8C00040FCD00126214A0240F806101800901E4DE868000603D52148286021482860E92E
:20F8E00060A869400706D416481E490160062141601D498160E10C0098FFF7F6FE00281496
:20F90000D10220E86000982861E86840210143E960FFF7E6FEA8683842FAD1E96802229118
:20F920001E43E9601421084000D0A960012E02D12068B8432060019880F3108803B0F0BDBE
:20F94000FD0014300040AAAA00000420024000F8FF00FF1F0000AAAAFD0020100240230170
:1CF960006745AB89EFCD55550000FF0F0000FFFF00000B214843401EFDD570479B
:00000001FF
